:100000000C942A090C9464090C9464090C946409F6
:100010000C9464090C9464090C9464090C946409AC
:100020000C9464090C9464090C9403360C94D9362E
:100030000C9445300C9464090C9464090C94640984
:100040000C9464090C9464090C9464090C9464097C
:100050000C94A3290C94CD300C9464090C9464097D
:100060000C9464090C9464090C9464090C9464095C
:100070000C9464090C9464090C9464090C9464094C
:100080000C9464090C9464090C9464090C9464093C
:100090000C9464090C94640996109610C210C21056
:1000A0002A115512551255124811E111F211F2118F
:1000B000B228B428B928BC28BF28C228C5288C2C4F
:1000C0007A2C932CE92B402D402D772C402D402D60
:1000D000C02C402DD42C202D402D402D402D402DC6
:1000E000F42C402D402DF12C402DAC2C402D402DDA
:1000F0003A2D3A2D3A2D3A2D3A2D3A2D3A2D3A2DC8
:100100003A2D3C2D402D8C2C6F2C402D402D402D18
:10011000402D402D402D402D402D402D402D3C2D7B
:10012000402D402D772C402D382D382D382D382D51
:10013000382D382D382D382D382D3C2D4A37713734
:10014000693871376938BD37E0376938373846382C
:1001500068747470733A2F2F716D6B2E666D2F015A
:10016000012800514D4B2069732074686520626539
:100170007374207468696E67206576657221002942
:10018000003A003B003C003D003E003F0040004183
:100190000042004300440045002A004C0049004B47
:1001A000004E0035001E001F002000210022002309
:1001B0000024002500260027002D002E00350053C6
:1001C000005400550048002B0014001A00080015C8
:1001D0000017001C0018000C00120013002F003044
:1001E0000031005F00600061005600390004001615
:1001F00000070009000A000B000D000E000F00337D
:10020000003400320028005C005D005E005700E111
:100210000064001D001B00060019000500110010FD
:1002200000360037003800E100520059005A005BE8
:10023000000100E000E300E200000000002C0000EC
:100240000000000000E2000151E700500051004FA3
:10025000006200630058000100010001000100017C
:100260000001000100010001000100010001000186
:10027000000100460047004A004D00010001000156
:100280000001000100010001000100010001000166
:1002900000010001000100C75CC65C010001000113
:1002A00000010001000100005C01000100010001EB
:1002B0000001000100010001000100C95CC85C01EF
:1002C0000001000100010001000100010001000126
:1002D000000100010001000100010001000100CB4C
:1002E0005CCA5C0100010001000100010001000185
:1002F00000010001000100010001000100010001F6
:1003000000A900C35CC45C01000100010001000100
:100310000000000000AE000000000000000100012D
:10032000000100AC00AA00AB000100010001004484
:10033000454255473A2064697361626C65642E0AD0
:100340000044454255473A20656E61626C65642EF3
:100350000A0000000000000000002A2B2800000016
:100360000000000000000000000000000029000064
:1003700000002C1E3420212224342627252E362D41
:100380003738271E1F202122232425263333362EDB
:1003900037381F0405060708090A0B0C0D0E0F104D
:1003A0001112131415161718191A1B1C1D2F313092
:1003B000232D350405060708090A0B0C0D0E0F1036
:1003C0001112131415161718191A1B1C1D2F313072
:1003D000354C00000000000000000000000000009C
:1003E000000000000000000000000000000000000D
:1003F0000000000000007E0F00D4FFFFFFC70000D8
:1004000000780A0025303258006C65645F746173AF
:100410006B3A20004F6E6573686F743A20616374A5
:100420006976653A2025640A000A00253033326C6B
:1004300062003A200025303258000A722F632030C3
:10044000313233343536373839414243444546300A
:100450003132333435363738394142434445460A20
:10046000007267626C696768742074696D657220D8
:1004700064697361626C652E0A007267626C6967F9
:1004800068742074696D657220656E61626C656464
:100490002E0A007267626C69676874207365742045
:1004A000687376205B4E4F454550524F4D5D3A2064
:1004B00025752C25752C25750A007267626C696795
:1004C00068742073657420687376205B45455052CC
:1004D0004F4D5D3A2025752C25752C25750A007227
:1004E00067626C69676874207261696E626F7720F9
:1004F000736574206873763A2025642C25642C2556
:10050000642C25750A007267626C696768742064E0
:10051000697361626C65205B4E4F454550524F4D8B
:100520005D3A207267626C696768745F636F6E66BC
:1005300069672E656E61626C65203D2025750A0035
:100540007267626C696768742064697361626C6564
:10055000205B454550524F4D5D3A207267626C6991
:100560006768745F636F6E6669672E656E61626C43
:1005700065203D2025750A007267626C69676874A2
:1005800020656E61626C65205B4E4F454550524F51
:100590004D5D3A207267626C696768745F636F6E65
:1005A0006669672E656E61626C65203D2025750A5F
:1005B000007267626C6967687420656E61626C6561
:1005C000205B454550524F4D5D3A207267626C6921
:1005D0006768745F636F6E6669672E656E61626CD3
:1005E00065203D2025750A007267626C6967687432
:1005F00020746F67676C65205B454550524F4D5DB9
:100600003A207267626C696768745F636F6E6669CF
:10061000672E656E61626C65203D2025750A00724B
:1006200067626C69676874206D6F6465205B4E4F0C
:10063000454550524F4D5D3A2025750A007267625C
:100640006C69676874206D6F6465205B4545505226
:100650004F4D5D3A2025750A007267626C696768C4
:10066000745F696E6974207267626C696768745F31
:10067000636F6E6669672E6D6F6465203D20302E56
:100680002057726974652064656661756C742076A4
:10069000616C75657320746F20454550524F4D2E27
:1006A0000A007267626C696768745F696E697420BA
:1006B0006565636F6E666967206973206E6F74206D
:1006C000656E61626C65642E0A007267626C6967B0
:1006D00068745F696E6974207374617274210A00B2
:1006E0007267626C696768745F696E6974206361C0
:1006F0006C6C65642E0A007267626C696768745F6F
:10070000636F6E6669672E7370656564203D202592
:10071000640A007267626C696768745F636F6E6613
:1007200069672E76616C203D2025640A007267623D
:100730006C696768745F636F6E6669672E73617456
:10074000203D2025640A007267626C696768745FE7
:10075000636F6E6669672E687565203D2025640AA3
:10076000007267686C696768745F636F6E6669675B
:100770002E6D6F6465203D2025640A007267626CEF
:10078000696768745F636F6E6669672E656E616224
:100790006C65203D2025640A007267626C69676899
:1007A000745F636F6E66696720454550524F4D3ADE
:1007B0000A0000047F3F1F643214643214783C1E28
:1007C0001E140A052223252628292A2C2D2F3032F3
:1007D000333536383A3B3D3E4042434547494A4C23
:1007E0004E5051535557595A5C5E60626466686951
:1007F0006B6D6F71737577797B7D7F818385878959
:100800008A8C8E90929496989A9C9E9FA1A3A5A75D
:10081000A8AAACAEAFB1B3B4B6B8B9BBBCBEBFC189
:10082000C2C3C5C6C7C9CACBCCCDCED0D1D2D2D314
:10083000D4D5D6D7D7D8D9D9DADADBDBDBDCDCDC28
:10084000DCDCDDDDDDDDDCDCDCDCDCDBDBDBDADAEB
:10085000D9D9D8D7D7D6D5D4D3D2D2D1D0CECDCC62
:10086000CBCAC9C7C6C5C3C2C1BFBEBCBBB9B8B677
:10087000B4B3B1AFAEACAAA8A7A5A3A19F9E9C9A02
:1008800098969492908E8C8A89878583817F7D7BD0
:1008900079777573716F6D6B6968666462605E5CB1
:1008A0005A5957555351504E4C4A49474543424077
:1008B0003E3D3B3A3836353332302F2D2C2A29280D
:1008C00026252322FFAA7F55406261636B6C69670E
:1008D000687420627265617468696E672064697308
:1008E00061626C650A006261636B6C6967687420A1
:1008F000627265617468696E6720656E61626C65BD
:100900000A006261636B6C6967687420627265617A
:100910007468696E6720746F67676C653A20257527
:100920000A006261636B6C69676874207374657038
:100930003A2025750A006261636B6C6967687420F0
:1009400064697361626C650A006261636B6C6967FC
:10095000687420656E61626C650A006261636B6C2D
:100960006967687420746F67676C653A2025750A3B
:10097000006261636B6C69676874206465637265AB
:100980006173653A2025750A006261636B6C696763
:10099000687420696E6372656173653A2025750A13
:1009A0000000000000000000000000000101020340
:1009B000040506080A0C0F1114181C2024292E33D4
:1009C000393F464C535B626A7179818A929AA2AA36
:1009D000B2B9C1C8CFD5DCE1E7EBF0F4F7FAFCFD22
:1009E000FEFFFEFDFCFAF7F4F0EBE7E1DCD5CFC843
:1009F000C1B9B2AAA29A928A8179716A625B534C98
:100A0000463F39332E2924201C1814110F0C0A08D4
:100A100006050403020101000000000000000000C0
:100A200000000101010101010101010202020202B3
:100A30000202020203030303030303030404040486
:100A4000040404050505050506060606060707074E
:100A5000070708080808090909090A0A0A0B0B0B05
:100A60000C0C0C0D0D0D0E0E0E0F0F0F10101111A2
:100A70001112121313141415151616171718181926
:100A8000191A1A1B1B1C1D1D1E1E1F20202122228D
:100A9000232424252626272829292A2B2C2D2D2ED0
:100AA0002F30313232333435363738393A3B3C3DEA
:100AB0003E3F404142434445464748494A4C4D4EDB
:100AC0004F50515354555658595A5B5D5E5F6162A1
:100AD00064656668696B6C6D6F7072737577787A30
:100AE0007B7D7E8082838587888A8C8E8F9193958B
:100AF00096989A9C9EA0A2A3A5A7A9ABADAFB1B3AF
:100B0000B5B7BABCBEC0C2C4C6C9CBCDCFD1D4D68E
:100B1000D8DBDDDFE2E4E7E9EBEEF0F3F5F8FAFD30
:100B2000FF3F00433E20004C25640A000A092D20A7
:100B3000537461747573202D0A686F73745F6B65ED
:100B400079626F6172645F6C65647328293A20254D
:100B50003032580A6B6579626F6172645F70726FD0
:100B6000746F636F6C3A20253032580A6B65796276
:100B70006F6172645F69646C653A20253032580A8F
:100B80006B65796D61705F636F6E6669672E6E6B02
:100B9000726F3A20253032580A74696D65725F723F
:100BA000656164333228293A202530386C580A00B0
:100BB0000A092D2056657273696F6E202D0A5649F9
:100BC000443A203078303444382868696E65796258
:100BD000757368206B6579626F6172647329205048
:100BE00049443A2030784543453828686263702983
:100BF000205645523A203078303030310A4255493B
:100C00004C443A2020284665622032372032303268
:100C100032290A4F5054494F4E533A204C554641C1
:100C20002045585452414B455920434F4E534F4C49
:100C30004520434F4D4D414E44204E4B524F20389E
:100C40003139320A4743433A20352E342E30204181
:100C500056522D4C4942433A20322E302E302041FC
:100C600056525F415243483A2061767235310A004C
:100C70000A092D20436F6E736F6C65202D0A455352
:100C8000432F713A09717569740A000A092D204DC4
:100C900061676963202D0A443A09446562756720DB
:100CA0004D65737361676520546F67676C650A589B
:100CB0003A094D6174726978204465627567204D08
:100CC0006F646520546F67676C65202D2053686FD3
:100CD00077206B65797072657373657320696E2018
:100CE0006D617472697820677269640A4B3A094BC6
:100CF0006579626F61726420446562756720546F24
:100D000067676C65202D2053686F77206B6579705D
:100D100072657373207265706F72740A4D3A09447C
:100D200065627567204D6F75736520546F67676CDA
:100D3000650A563A0956657273696F6E0A533A0925
:100D40005374617475730A433A0941637469766137
:100D5000746520436F6E736F6C65204D6F64650A18
:100D600046312D4631303A095377697463682074EF
:100D70006F204C6179657220302D39202846313042
:100D8000203D204C30290A302D393A0953776974B7
:100D9000636820746F204C6179657220302D390AA8
:100DA00047524156453A0953776974636820746F16
:100DB000204C6179657220302028616C7465726EF8
:100DC000617465290A423A094A756D7020746F2072
:100DD000426F6F746C6F616465720A4553433A09E0
:100DE0004A756D7020746F20426F6F746C6F616410
:100DF00065722028616C7465726E617465290A459C
:100E00003A095072696E7420454550524F4D205337
:100E1000657474696E67730A4253504143453A09D9
:100E2000436C65617220454550524F4D0A4E3A0958
:100E30004E4B524F20546F67676C650A00626163C6
:100E40006B6C696768745F636F6E6669672E726149
:100E5000773A20253032580A2E656E61626C653A09
:100E60002025750A2E6C6576656C3A2025750A007A
:100E70006B65796D61705F636F6E6669672E726115
:100E8000773A20253032580A2E737761705F636F8E
:100E90006E74726F6C5F636170736C6F636B3A201A
:100EA00025750A2E636170736C6F636B5F746F5F7F
:100EB000636F6E74726F6C3A2025750A2E737761BA
:100EC000705F6C63746C5F6C6775693A2025750A96
:100ED0002E737761705F7263746C5F726775693AC5
:100EE0002025750A2E737761705F6C616C745F6C7E
:100EF0006775693A2025750A2E737761705F726194
:100F00006C745F726775693A2025750A2E6E6F5F83
:100F10006775693A2025750A2E737761705F67726D
:100F20006176655F6573633A2025750A2E73776174
:100F3000705F6261636B736C6173685F6261636B46
:100F400073706163653A2025750A2E6E6B726F3A75
:100F50002025750A0064656275675F636F6E666958
:100F6000672E7261773A20253032580A2E656E61FD
:100F7000626C653A2025750A2E6D61747269783A43
:100F80002025750A2E6B6579626F6172643A20259F
:100F9000750A2E6D6F7573653A2025750A006565B3
:100FA000636F6E6669673A0A64656661756C745F43
:100FB0006C617965723A2025750A003F004E4B52EC
:100FC0004F3A206F66660A004E4B524F3A206F6EC2
:100FD0000A000A6D6F7573653A206F66660A000A2B
:100FE0006D6F7573653A206F6E0A000A6B657962E2
:100FF0006F6172643A206F66660A000A6B657962F7
:101000006F6172643A206F6E0A000A6D61747269D2
:10101000783A206F66660A000A6D61747269783AE0
:10102000206F6E0A000A64656275673A206F666613
:101030000A000A64656275673A206F6E0A000A0A40
:101040004A756D70696E6720746F20626F6F746C83
:101050006F616465722E2E2E2000433E2000436C8B
:10106000656172696E6720454550524F4D0A000A0E
:10107000002530325820006B6579626F6172645FC1
:101080007265706F72743A200064656C5F6B65798D
:101090005F6269743A2063616E27742064656C3AFC
:1010A00020253032580A006164645F6B65795F62A5
:1010B00069743A2063616E2774206164643A202564
:1010C0003032580A005B735D005B575D005B535D17
:1010D000005B525D005B445D005B435D000A03689A
:1010E0000062006300700000002803680069006E61
:1010F0000065007900620075007300680020006BD5
:10110000006500790062006F006100720064007386
:101110000000000403090409025B00030100A0FAB7
:10112000090400000103010100092111010001224D
:1011300040000705810308000109040100010300C4
:101140000000092111010001226D00070582032022
:10115000000109040200020300000009211101003E
:101160000122220007058303200001070503032055
:1011700000011201000200000008D804E8EC0100A0
:10118000010200010631FF0974A10109751500264D
:10119000FF009520750881020976150026FF00954D
:1011A0002075089102C005010980A101850319017C
:1011B0002AB700150126B700950175108100C005FA
:1011C0000C0901A101850419012AA002150126A01C
:1011D00002950175108100C005010906A10185066F
:1011E000050719E029E71500250195087501810219
:1011F0000507190029EF1500250195F075018102F9
:1012000005081901290595057501910295017503D8
:101210009101C005010906A101050719E029E7159B
:101220000025019508750181029501750881010568
:1012300007190029FF150026FF0095067508810093
:101240000508190129059505750191029501750398
:101250009101C00011241FBECFEFD0E2DEBFCDBF91
:1012600004B603FE18C08091BE039091BF03A09105
:10127000C003B091C1038730904BA740B04B59F4E5
:101280001092BE031092BF031092C0031092C103CC
:10129000E0E0F0EF099511E0A0E0B1E0ECE5F3E764
:1012A00000E00BBF02C007900D92A43DB107D9F733
:1012B00023E0A4EDB1E001C01D92AE3BB207E1F71F
:1012C0000E94F11D0C94AC390C940000FF93EF9335
:1012D000E091D401F091D501309709F00995EF9193
:1012E000FF910895FC018591803011F0EFDFFBCF75
:1012F0000895FF27E0E230E247FF0CC0419597FFD9
:1013000009C0EDE26095709580959095611D711D05
:10131000811D911D27FF02C0219530E350E2AA27CD
:10132000660F771F881F991FAA1FA41710F0A41B10
:1013300063955A95A9F7AA3008F0A95FA05DAF930D
:10134000F395611571058105910541F7ED3211F4B1
:10135000EF93F395F21718F43F93F395FBCF8F912A
:10136000B5DFFA95E1F70895E991F991859180301B
:1013700021F0853219F0AADFF9CF089520E0E89432
:1013800055915532C1F3503311F4689455915A3345
:1013900048F4505390F3220F022E220F220F200DFB
:1013A000250FF4CF0EF4219589919991533619F3B5
:1013B000533729F1533559F1BC0188279927E8940F
:1013C0005C3621F48991999168945591543639F499
:1013D00046EF7EF077FF0DC08FEF9FEF0AC05537C5
:1013E0004AE039F0583540E121F0523642E009F048
:1013F0000895FF93EF937DDFEF91FF91B7CFFF93B8
:10140000EF93FC0181918030B9F360DFFBCFFF9354
:10141000EF9368DFF1CFDF93CF93CDB7DEB725969B
:10142000A3DFCF91DF910895E82FF0E0E85CFE4F55
:101430008081E82FE295EF70F0E031A1282F2F7026
:1014400081E090E001C0880F2A95EAF7932F982B4E
:1014500091A392A18095892382A30895E82FF0E0BB
:10146000E85CFE4F8081E82FE295EF70F0E031A15B
:10147000282F2F7081E090E001C0880F2A95EAF7AD
:10148000982F9095932391A392A1892B82A30895DD
:101490004F925F926F927F928F929F92AF92BF9284
:1014A000CF92DF92EF92FF921F93CF93DF93162F8D
:1014B000EC0124E0629FC00DD11D1124C880D980A9
:1014C000EA80FB80188219821A821B82862F0E9472
:1014D000140A0E94711DE6E2F1E020E030E0812C68
:1014E000912C540183944191A42FA295AF70B0E048
:1014F00090968C91488059806A807B8090E04F70F4
:10150000DC0102C0B595A7954A95E2F7A0FD0BC096
:10151000D501C401022E04C0880F991FAA1FBB1F4A
:101520000A94D2F703C080E090E0DC018429952979
:10153000A629B72988839983AA83BB832F5F3F4F4E
:101540002231310581F6812F0E942E0A81E04881E7
:1015500059816A817B814C155D056E057F0509F413
:1015600080E0DF91CF911F91FF90EF90DF90CF90BF
:10157000BF90AF909F908F907F906F905F904F90B3
:101580000895E82FF0E0EA5DFE4F8081E82FE295B4
:10159000EF70F0E031A1282F2F7081E090E001C0C2
:1015A000880F2A95EAF7932F982B91A392A1809503
:1015B000892382A30895E82FF0E0EA5DFE4F808141
:1015C000E82FE295EF70F0E031A1282F2F7081E035
:1015D00090E001C0880F2A95EAF7982F9095932301
:1015E00091A392A1892B82A308956F927F928F92EB
:1015F0009F92AF92BF92CF92DF92EF92FF920F93A2
:101600001F93CF93DF93182FD92FC62F862F0E94B9
:10161000C10A0E94711D41E050E060E070E00C2EB4
:1016200004C0440F551F661F771F0A94D2F728E3A2
:10163000622E21E0722EE12FFD2F9F01285E3F4F89
:10164000D0E08F0180809180A280B380D3018D9102
:101650003D01E82EE2949FE0E922F12CD70190961B
:10166000EC90F12C8F70D70102C0B595A7958A95A3
:10167000E2F7A0FD0AC075016401C42AD52AE62A52
:10168000F72AC082D182E282F3823496D801CD90CB
:10169000DD90ED90FC908C149D04AE04BF0409F025
:1016A000D1E0E217F30769F68C2F0E94DB0A8D2F39
:1016B000DF91CF911F910F91FF90EF90DF90CF902E
:1016C000BF90AF909F908F907F906F900895CF9331
:1016D000DF93A8E3B1E04EE351E061E070E08D916B
:1016E000E82FE295EF70F0E021A18F70EB0102C0CE
:1016F000CC0FDD1F8A95E2F7CE019C2F90959223A7
:1017000091A392A1892B82A34A175B0741F7DF912E
:10171000CF910895CF93DF93A6E2B1E048E351E083
:1017200061E070E08D91E82FE295EF70F0E021A18B
:101730008F70EB0102C0CC0FDD1F8A95E2F7CE015E
:101740009C2F9095922391A392A1892B82A34A1753
:101750005B0741F7DF91CF9108950E94670B0C94CE
:101760008A0B0C94AD0B8F929F92AF92BF92CF9247
:10177000DF92EF92FF920F931F93CF93DF93F82E98
:10178000092FC82FD92F86EDA82E81E0B82E45014C
:10179000CF2CD92E10E0F60181919191A191B191B8
:1017A0006F01F40181939193A193B1934F01612F44
:1017B0008F2D902F0E94480A1F5F163061F710E0AE
:1017C000612F8F2D902F0E94F50A1F5F1231C1F7F4
:1017D0002EEE31E080E0F501C190D190E190F190E2
:1017E0005F014991599169917991C416D506E60630
:1017F000F70609F081E02A153B0569F7DF91CF91E3
:101800001F910F91FF90EF90DF90CF90BF90AF901E
:101810009F908F9008950E944E2440E86FEF80E0E3
:101820000E94A5218BE00E944B2460E070E0CB0178
:101830000E9462190C946E19CF93C82F2BE533E0E8
:1018400081FF06C048E760E080E00E94A71E05C057
:1018500040E060E080E00E94B51E2EE533E0C0FF6E
:1018600006C048E760E080E00E94A71E05C040E097
:1018700060E080E00E94B51E21E633E0C2FF06C0B2
:1018800048E760E080E00E94A71E05C040E060E0FD
:1018900080E00E94B51ECF910C94AE1F68E183E0FA
:1018A0000E94931E87E00E941C0C2FEF85EA9EE0A9
:1018B000215080409040E1F700C0000080E00C948F
:1018C0001C0C873A2DE5920721F0883A9D4541F09E
:1018D0000FC0FB018281882359F083E691E006C0A6
:1018E000FB018281882321F080E591E00E943B0E7C
:1018F00081E0089581E008950C94610C08950C94A2
:101900007E0C1F93CF93DF9300D000D01F92CDB7F2
:10191000DEB749835A836B833091EF0189819A81C5
:10192000311114C0662359F0222349F00E948E140D
:10193000182F682F89819A810E94371403C00E9452
:101940006214182F69817A81812F04C00E948E143D
:1019500069817A810F900F900F900F900F90DF9117
:10196000CF911F910C94EF1BFC01262F40815181D8
:101970006281738184810C94810C81E00895CF93FE
:10198000DF93EC0160E00E94B40CBE01DF91CF91C7
:101990000C947F0C0C947C1D0C94781D08950E946F
:1019A000E1120E94CE0C2FEF84E39CE02150804096
:1019B0009040E1F700C000000C94F3300F931F93A8
:1019C000CF93DF938C0161E00E94B40CEC01B8016D
:1019D0000E947C0C882369F1B801CE010E94A328E3
:1019E000882339F1B801CE010E943F2E882309F1E6
:1019F000B801CE010E946E2A8823D9F0B801CE0129
:101A00000E949B2D8823A9F0B801CE010E942026B8
:101A1000882379F0F80182818823E1F1CF3D8CE5BC
:101A2000D80781F160F4C115FCE5DF0721F40E94BD
:101A3000CF0CC0E036C0C130DC4579F02BC0CC35CE
:101A4000EDE5DE0729F1CD35FDE5DF07F1F0CB351A
:101A5000DD4501F50E9425191DC08091DA02C82FCD
:101A6000C095C170C0FB80F98093DA02CC2329F0C5
:101A700081E493E00E947209DCCF8FE293E00E9440
:101A800072090FC00E94D219D4CF0E941C1902C043
:101A90000E942819C801DF91CF911F910F910C94DA
:101AA0007A0C8C2FDF91CF911F910F9108950E9496
:101AB000253080E00E945B290E949E0E0C946125D7
:101AC0000E945B270E94A10E0E94EC240C942B30F4
:101AD000DF92EF92FF920F931F93CF93DF93E82F44
:101AE000F0E0EE5AFC4FD490282F269526952695A7
:101AF00030E0F901EE50FC4F0491877010E0082EA1
:101B000002C0159507950A94E2F701701127F901B3
:101B1000EE51FC4FE490F12C082E02C0F594E794AE
:101B20000A94E2F791E0E922FF24F901EE52FC4F1A
:101B3000C491D0E002C0D595C7958A95E2F7C170EF
:101B4000DD270115110519F081EE0E94270FE11420
:101B5000F10419F086EE0E94270F8D2D0E9444108B
:101B6000EF2819F086EE0E94CE0F012B19F081EEBE
:101B70000E94CE0FCD2B51F08CE2DF91CF911F91BF
:101B80000F91FF90EF90DF900C944410DF91CF9174
:101B90001F910F91FF90EF90DF900895EF92FF92C9
:101BA0000F931F93CF93DF938C01F62E8AE0E82EDC
:101BB000F8018491882309F457C0813009F042C0AC
:101BC000E8012196FE018491813031F42196FE01D5
:101BD00084910E94441039C0823039F4E801229681
:101BE000FE0184910E94270F30C0833039F4E80150
:101BF0002296FE0184910E94CE0F27C0843029F5E1
:101C0000E8012296FE01249180E090E030E020532C
:101C100031092A30310560F4E89EA001E99E500D9B
:101C20001124C901840F951F2196FE012491EECF46
:101C3000009759F0EFE9FFE03197F1F700C000009D
:101C40000197F6CF0E94680DE8018E010F5F1F4FCC
:101C50008F2D882309F4ACCFEFE9FFE03197F1F73E
:101C600000C000008150F5CFDF91CF911F910F91FF
:101C7000FF90EF90089560E00C94CE0D8295982F20
:101C8000937344E0949F900111248C7C86958695F3
:101C9000282B822F8575880F2A7A2695822B089506
:101CA000CF93DF93D92F0E943E0EC82F8D2F0E9415
:101CB0003E0E2C2F30E0322F2227A901482BCA01DB
:101CC000DF91CF910895CF92DF92EF92FF920F9321
:101CD0001F93CF93DF936B017C01CB010E94500EC9
:101CE000EC01C7010E94500EAC01CE01A0E0B0E0B3
:101CF000DC019927882760E070E08C019D01042BAE
:101D0000152B262B372BC901B801DF91CF911F91DD
:101D10000F91FF90EF90DF90CF9008950C941C0CE2
:101D200081E008950C94900E0895CF93C82F0E94DF
:101D30008E0E8C2F0E94920ECF91089580E00C940D
:101D4000950E0E949B2E0C94950ECF930E949B2E75
:101D5000C82F8091EE01C81741F1C093EE01809128
:101D6000DA0282FF1EC080FF04C089E094E00E9476
:101D700072098091DA0280FF0CC01F92CF9384E039
:101D800094E09F938F930E940B0A0F900F900F90F7
:101D90000F908091DA0280FF04C082E094E00E94FC
:101DA00072098C2FCF910C94950ECF910895CF93FB
:101DB000DF93CDB7DEB72B970FB6F894DEBF0FBE1B
:101DC000CDBF4F83588769877A878B8761110E94BF
:101DD00054189E012F5F3F4F86E0F90111928A95BA
:101DE000E9F785E0FE013796D90101900D928A95B9
:101DF000E1F789819A814C815D81452B31F09F3FCC
:101E000031F491E08F3F19F403C091E001C090E0FC
:101E100090FF09C049815A816B817C818D819E81AF
:101E20000E94751705C0C9010E94BD0C8111F2CF37
:101E30002B960FB6F894DEBF0FBECDBFDF91CF91CA
:101E40000895FC01808191810E94D0140895CF9360
:101E5000882309F4A1C0C82F8238C1F40E949B2EA8
:101E600081FD9AC069E380910201909103010E9473
:101E7000E02F0E9476182FEF81EE94E021508040F1
:101E80009040E1F700C0000069E319C0833801F514
:101E90000E949B2E80FD80C063E58091020190919D
:101EA00003010E94E02F0E9476182FEF81EE94E04C
:101EB000215080409040E1F700C0000063E5809130
:101EC0000201909103010E94EB2FCF910C947618A0
:101ED0008438C1F40E949B2E82FD5EC067E480912D
:101EE0000201909103010E94E02F0E9476182FEFCB
:101EF00081EE94E0215080409040E1F700C0000066
:101F000067E4DDCF8CEF8C0F813AF8F48C2F0E94C0
:101F1000522D811141C06C2F8091020190910301DB
:101F20000E943E2F882349F06C2F809102019091EE
:101F300003010E94EB2F0E9476186C2F8091020102
:101F4000909103010E94E02FC0CF80E28C0F883077
:101F500048F4C77081E001C0880FCA95EAF70E9473
:101F60003718B3CFEBE5EC0FE33040F4F0E0E45981
:101F7000FE4F808190E0CF910C94FC2EC85AC7315F
:101F800058F4EC2FF0E0EE0FFF1FE25CFE4F808173
:101F90009181CF910C94122FCF910895882309F449
:101FA0005BC0682F823879F40E949B2E81FF54C059
:101FB00069E380910201909103010E94E02F0E9449
:101FC000761869E310C08338B1F40E949B2E80FF1D
:101FD00043C063E580910201909103010E94E02FCC
:101FE0000E94761863E580910201909103010E949E
:101FF000EB2F0C947618843879F40E949B2E82FF84
:102000002BC067E480910201909103010E94E02FB0
:102010000E94761867E4E7CF8CEF860F813A18F3B9
:1020200080E2860F883048F4677081E001C0880F35
:102030006A95EAF70E943D18DCCF8BE5860F833066
:1020400020F480E090E00C94FC2E685A673120F474
:1020500080E090E00C94122F08951F93CF93DF93AC
:10206000182FEB010E94270F209741F08FE99FE086
:102070000197F1F700C000002197F6CF812FDF9183
:10208000CF911F910C94CE0F893319F060E070E06E
:1020900002C060E570E00C942D10882321F00E94AE
:1020A00037180C9476180895882321F00E943D1863
:1020B0000C9476180895CF92DF92EF92FF920F93CF
:1020C0001F93CF93DF937C01D62FC72FFC01128182
:1020D000058102950F700E942D188823B9F01123F5
:1020E000A9F08C2F807F803421F080E28D0F883022
:1020F00068F08091250382FD09C082E00E94D61815
:102100000E942D1891E0D82ED92601C0D12CCC2EBA
:10211000C2948FE0C8228C2D90E08C30910508F09D
:10212000C4C1FC01E45BFF4F0C9410398C2F807FFD
:10213000CF70882311F0C295C07F112399F0CC2372
:1021400009F49FC180E28D0F883010F0D11104C0D6
:102150008C2F0E94371803C08C2F0E9447180E94B2
:1021600076188FC18D2F0E94CE0FCC2309F49DC10C
:1021700080E28D0F883038F1DD2329F18C2F0E9409
:102180004D1824C08C2F807FCF70803211F0C29503
:10219000C07FDD2319F0D130A1F13DC0809125032E
:1021A00082FF17C0112349F0CC2329F08C2F0E9405
:1021B00037180E94761880E065C180E00E94CE0F3B
:1021C000CC2309F472C18C2F0E943D180E9476180E
:1021D0006CC1112371F0002341F0013031F40E94F1
:1021E00057188C2B0E945F1860C10E9457188C2BC7
:1021F0001DC0002319F0013009F457C10E946C186A
:1022000025C0112321F0063008F04FC10EC0053063
:1022100008F04BC11BC0112361F0002331F0F7011E
:10222000858180FF2EC18F7085838C2F0E944D1079
:102230003CC1002359F0D93309F034C1FFEF07EE58
:1022400013E0F15000401040E1F72AC18C2F0E94AA
:1022500054102BC18C2F86958695837019F0813090
:1022600061F023C1112321F08D2F9C2F937002C0A8
:1022700080E090E00E94FC2E20C1112321F08D2FE0
:102280009C2F937002C080E090E00E94122F15C135
:102290008C2F837009F047C011110BC12D2F22958F
:1022A00026952770220F220F6D2F6F70862F90E0DA
:1022B000A0E0B0E0022E04C0880F991FAA1FBB1F28
:1022C0000A94D2F7D4FF10C04FE050E060E070E015
:1022D00004C0440F551F661F771F2A95D2F74095FB
:1022E00050956095709503C040E050E0BA01C695E6
:1022F000C695C3708A019B01082B192B2A2B3B2BF7
:10230000C901B801C23049F058F4C13019F00E9437
:102310004D13CFC00E943B13CCC00E945F13C9C0B5
:102320000E943913C6C0112319F08C2F817001C08F
:102330008695882309F4BDC02D2F229526952770F8
:10234000220F220F6D2F6F70862F90E0A0E0B0E07B
:10235000022E04C0880F991FAA1FBB1F0A94D2F730
:10236000D4FF10C04FE050E060E070E004C0440FC4
:10237000551F661F771F2A95D2F740955095609597
:10238000709503C040E050E0BA01C695C695C37091
:102390008A019B01082B192B2A2B3B2BC901B80161
:1023A000C23049F058F4C13019F00E94121481C0B3
:1023B0000E9400147EC00E9424147BC00E947313EC
:1023C00078C0CF70112339F08C2F0E9499138D2F74
:1023D0000E944D106EC08D2F0E9454108C2F0E94B1
:1023E000BA1367C0D23F21F128F4D03F41F0D13F6A
:1023F000C1F043C0D33F19F1D43F79F03EC011235F
:1024000041F0053008F051C08C2F8F710E94DF130E
:102410004CC0063008F049C0F7CF8091250382FFF9
:1024200018C0112339F08C2F8F710E9499133DC071
:102430001123C9F38C2F8F710E94BA1336C0112358
:1024400029F08C2F8F710E9484132FC00E947F135C
:102450002CC0112349F0CF718C2F0E94991363E097
:102460008C2F0E94BB1821C081E00E94D618023038
:10247000E0F082E00E94D61818C0112331F000234A
:1024800091F28D2F0E94270F10C0002399F2D933AB
:1024900049F41FEF27EE33E0115020403040E1F7C0
:1024A00000C000008D2F0E94CE0F88EF8C0D84306D
:1024B00020F40E949B2E0E94950EDD20C9F00E9400
:1024C000291880FD15C0F70112820E9423180E946E
:1024D0009913C7010E9499120E942318DF91CF918E
:1024E0001F910F91FF90EF90DF90CF900C94BA1353
:1024F000DF91CF911F910F91FF90EF90DF90CF90E0
:1025000008950F931F93CF93DF93EC016881798136
:102510008A810E94DB148C010E9436140E942713CA
:10252000B801CE010E945B10DF91CF911F910F91F6
:102530000895CF93DF93EC01988189812B813C81B1
:10254000232B31F08F3F31F481E09F3F19F403C01A
:1025500081E001C080E080FD1DC0CE010E94DE0C44
:10256000811110C00E942D188823A1F08A81882330
:1025700089F08091250382FD0DC082E0DF91CF912B
:102580000C94D618CE010E948112CE01DF91CF911A
:102590000C94BF0CDF91CF91089580E090E00E94F1
:1025A000FC2E80E090E00E94122F0E9454180C94A0
:1025B000761880910201909103010E94F62F0C94ED
:1025C000CD120E9444180C94D91292959F709630A7
:1025D00079F010F4925001C09A50923068F4803F24
:1025E00069F018F4883E40F409C0843F29F406C01D
:1025F000883E20F0813F11F080E0089581E0089549
:10260000FC01808191810E94D0140E94E5120895FE
:10261000CF93DF9300D000D01F92CDB7DEB70F90DD
:102620000F900F900F900F90DF91CF910895CF935F
:10263000DF9300D000D000D0CDB7DEB726960FB61E
:10264000F894DEBF0FBECDBFDF91CF9108950895FE
:1026500008950C9428130C9429130E942B13609353
:102660003A0270933B0280933C0290933D020C949B
:10267000CD120C942D130F931F9300913A021091D9
:102680003B0220913C0230913D02602B712B822B4A
:10269000932B1F910F910C942D130F931F93009167
:1026A0003A0210913B0220913C0230913D0260239E
:1026B0007123822393231F910F910C942D130F9359
:1026C0001F9300913A0210913B0220913C023091FD
:1026D0003D0260277127822793271F910F910C9449
:1026E0002D130C9428130E9471136093360270937B
:1026F000370280933802909339020C94CD1260E037
:1027000070E0CB010C9473130F931F9341E050E0E2
:1027100060E070E08A019B0104C0000F111F221FBE
:10272000331F8A95D2F7C901B8011F910F910C94FC
:1027300073130F931F9341E050E060E070E004C01A
:10274000440F551F661F771F8A95D2F78091360276
:1027500090913702A0913802B09139028A019B0111
:10276000082B192B2A2B3B2BC901B8011F910F9164
:102770000C9473130F931F9341E050E060E070E0FE
:1027800004C0440F551F661F771F8A95D2F74095E6
:102790005095609570958091360290913702A09186
:1027A0003802B09139028A019B01082319232A2398
:1027B0003B23C901B8011F910F910C9473130F9320
:1027C0001F9341E050E060E070E004C0440F551FEB
:1027D000661F771F8A95D2F7809136029091370253
:1027E000A0913802B09139028A019B01082719276C
:1027F0002A273B27C901B8011F910F910C9473132D
:102800000F931F93009136021091370220913802E6
:1028100030913902602B712B822B932B1F910F91DA
:102820000C9473130F931F9300913602109137028B
:10283000209138023091390260237123822393233F
:102840001F910F910C9473130F931F9300913602F5
:102850001091370220913802309139026027712798
:10286000822793271F910F910C947313089522E1EF
:10287000929F800D1124E82FE695E695E6958770E6
:1028800051E001C0550F8A95EAF785E0E89FF00115
:102890001124E051FE4F20E030E070E04081CB0198
:1028A000022E02C0969587950A94E2F78170819571
:1028B00084278523842781932F5F3F4F253031055F
:1028C00069F7089522E1929F800D1124682F669583
:1028D00066956695982F977085E0689FB0011124E2
:1028E00040E050E080E0FB01E40FF51FE051FE4FB7
:1028F000208130E0092E02C0369527950A94E2F730
:1029000021703327042E01C0220F0A94EAF7822B8C
:102910004F5F5F4F4530510531F70895BF92CF9219
:10292000DF92EF92FF920F931F93CF93DF938C016F
:10293000C0903602D0903702E0903802F090390211
:1029400080913A0290913B02A0913C02B0913D02ED
:10295000C82AD92AEA2AFB2ACFE1D0E0D701C6014A
:102960000C2E04C0B695A795979587950A94D2F733
:1029700080FD04C0219790F7B12C07C0BC2EB80190
:102980008C2F0E94021C0197A9F38B2DDF91CF9110
:102990001F910F91FF90EF90DF90CF90BF9008951F
:1029A000CF93DF93EC010E948E14BE010E94021CA3
:1029B000DF91CF9108951F93CF93DF93EB01909117
:1029C000EF01992321F0CB010E94D01413C088237A
:1029D00049F0CB010E948E14182F682FCE010E945F
:1029E000371404C0CB010E946214182FBE01812F3E
:1029F0000E94021CDF91CF911F9108951F93CF93E6
:102A0000DF93C0913E0216E080913F02C81799F013
:102A1000D0E01C9FF0011D9FF00D1124E05CFD4FE4
:102A20004081518162817381848195810E94171355
:102A30002196C770E9CFDF91CF911F910895409102
:102A400070025091710260917202709173028091D4
:102A50007402909175020C941713EF92FF920F93EA
:102A60001F93CF93DF938091750282958F7009F049
:102A700065C080917202882309F460C080913E0293
:102A8000F0903F0210917002009171026091730208
:102A90007091740291E01F3F09F090E0C091000135
:102AA000D0910101292F96E0E92E8F1509F446C037
:102AB0006115710521F00F3F21F030E003C031E0D6
:102AC00001C0322F90E030FD36C0E89EF001E99E53
:102AD000F00D1124DF01A05CBD4F11963C911197C0
:102AE000301329C03C91311326C012963C911297A5
:102AF000311121C013964D915C911497461B570BD1
:102B00004C175D07C0F4809175028F7080618093CF
:102B10007502EB5BFD4F80818F708061808380E761
:102B200092E00E949912DF91CF911F910F91FF9037
:102B3000EF900C94FE1401968770B7CFDF91CF9180
:102B40001F910F91FF90EF9008959F92AF92BF92C7
:102B5000CF92DF92EF92FF920F931F93CF93DF9369
:102B6000CDB7DEB761970FB6F894DEBF0FBECDBF0D
:102B70008C0185E0F801DE011D9601900D928A9589
:102B8000E1F7D8011296EC9090917002E0917102F9
:102B900020917302309174022115310531F0EF3F1D
:102BA00031F481E09F3F19F403C081E001C080E06F
:102BB000B82FB1709B2E80FD47C1D8014C91119662
:102BC0005C9111971396AD90BC90149780E7C82E36
:102BD00082E0D82EF0907202B501621B730B209137
:102BE000000130910101FF2009F4D9C080917502E4
:102BF0006217730708F095C0282F207F09F052C094
:102C00005E1313C0491311C0FE2CE1100EC08F706B
:102C10008061809375020E941F15C6010E9499125F
:102C200080917502F80185834DC1AB2831F05F3F7B
:102C300031F481E04F3F19F403C081E001C080E02E
:102C400080FD03C081E08E2502C080E090E0F82F77
:102C5000F170FF2E80FF1CC080913E0220913F0248
:102C600036E0821709F40BC190E0389FF001399FDC
:102C7000F00D1124E05CFD4F6181561306C06081A8
:102C8000461303C06281E61203C001968770E9CF44
:102C9000FE2CEE2009F416C18091750281608093AC
:102CA000750254C05E1306C0491304C0E11002C08F
:102CB000F80199C0C8010E940013882361F1EE2039
:102CC00051F120917502822F82958F7090E00297CA
:102CD00074F0809170029091710298878F831986A9
:102CE000BB86AA862C87CE0107960E94991286E0A1
:102CF000F801A0E7B2E001900D928A95E1F70E94F9
:102D00002D150E941F150AC05E1711F1C8010E94FF
:102D1000001381112CC0C8010E949912FF24F39462
:102D2000D1C0282F207F81F77A2DB98AA88A6E2DED
:102D300089890E94081380E792E00E94991286E038
:102D4000D6011D928A95E9F70E941F15F12CBAC091
:102D50004913DCCFE110DACFF8018583C8010E9466
:102D6000991286E0D6011D928A95E9F7ABC0EE2054
:102D700091F220917502822F82958F7090E00297D8
:102D80000CF4B5CF80917002909171029A8389837F
:102D90001B82BD82AC822E83CE010196A6CF621724
:102DA000730708F044C0FE2CEE2009F4B4CF5E1384
:102DB00030C049132EC02091750220FD21C0822F02
:102DC00082958F70482F50E041155105C9F0F801E8
:102DD00025834F30510541F08F5F982F9295907F5A
:102DE000822F8F70892B8583C8010E94991286E0FB
:102DF000F801A0E7B2E001900D928A95E1F73CC09E
:102E000086E0F801A0E7B2E001900D928A95E1F723
:102E100059C0C8010E940013811169CF80917502C9
:102E2000816080937502C8010E9499124BC07A2D6F
:102E3000B98AA88A6E2D89890E94081386E0D60176
:102E40001D928A95E9F718C0EE2009F464CFC801F5
:102E50000E940013F82E882309F45DCF86E0F80164
:102E6000A0E7B2E001900D928A95E1F780E792E049
:102E70000E94210F0E942D150E941F1523C04D870F
:102E80005E878D859E850E94D014292F22952F70F4
:102E9000223028F49F7039F0811105C00BC0243016
:102EA00028F49F7049F4805E883020F0C8010E94A9
:102EB00099129F2CF92C06C0D80115969C91907FF1
:102EC00091F7F8CF8F2D61960FB6F894DEBF0FBE45
:102ED000CDBFDF91CF911F910F91FF90EF90DF90C9
:102EE000CF90BF90AF909F9008951F93CF93DF93A3
:102EF000CDB7DEB72C970FB6F894DEBF0FBECDBFAF
:102F00004F83588769877A878B879C87CE0107967E
:102F10000E94A5158823D1F09F8188852A853B854D
:102F2000232B31F08F3F31F481E09F3F19F403C030
:102F300081E001C080E080FD47C04F8158856985F0
:102F40007A858B859C850E9417133EC086E0FE0122
:102F50003796DE01119601900D928A95E1F7FF8177
:102F6000E8856A857B856115710531F0EF3F31F4A5
:102F700081E0FF3F19F403C081E001C080E080FDE3
:102F800023C020913F0230E0C90101968770992744
:102F900040913E0250E084179507F1F1F983EA83EE
:102FA0007D836C8396E0929FD001939FB00D112496
:102FB000A05CBD4FFE01319601900D929A95E1F70C
:102FC00080933F020E94FE1416E080913E02909191
:102FD0003F02891771F1189FC0011124805C9D4F39
:102FE0000E94A515882329F1E0913E021E9FF00161
:102FF0001124E05CFD4F40815181628173818481A5
:1030000095810E94171380913E0290E0019687708F
:10301000992780933E02D9CF0E94E11210923F027D
:1030200010923E02E0E7F2E086E0DF011D928A9511
:10303000E9F72C960FB6F894DEBF0FBECDBFDF9137
:10304000CF911F91089580919602859585958595DC
:1030500008958091960287700895909196029770D6
:1030600081E009F480E008958091B902089590917B
:10307000B902892B8093B902089580959091B90285
:1030800089238093B90208951092B902089590910E
:10309000B802892B8093B802089580959091B80268
:1030A00089238093B80208951092B8020895809100
:1030B0009702089508950C945A180C945B189091F7
:1030C000250392FD08C090919702981721F08093F4
:1030D00097020C945D18089580919702882329F037
:1030E0001092970280E00C945D180895CF93DF93BF
:1030F000E0910201F09103018091B9028083E09197
:103100000201F091030190818091B802892B8083A4
:1031100080919702882381F0E0910201F0910301F0
:103120009081892B808380910201909103010E94FC
:10313000282F81110E946C18C0910201D0910301C7
:1031400040E250E066E772E0CE010E945739892BD9
:1031500069F080E2FE01A6E7B2E001900D928A9547
:10316000E1F7CE01DF91CF910C94A72EDF91CF91A3
:1031700008950C945A189091250392FD10C098E080
:10318000899F90011124262B209396020E94991367
:10319000809196028595859585950C94B9180C9427
:1031A00099131092960280E00C94B918209196021F
:1031B0008095822380939602982F977099F430E03F
:1031C000482F082E000C550B2417350759F0909105
:1031D000250392FD07C08595859585950E94BA13B4
:1031E0000C94D1180895CF939091250392FB222738
:1031F00020F92817F9F0C82F892FC0FB82F9809396
:10320000250380912403909125030E94551982E0A3
:103210000E94D6188091DA0280FF0CC01F92CF93D3
:1032200084E194E09F938F930E940B0A0F900F907C
:103230000F900F90CF9108958091250382FB8827EE
:1032400080F991E089270C94F31881E00C94F3182D
:1032500080E00C94F3186FEF7FEF80E090E00C9427
:10326000963980E090E00E94723921E0893E9E4FBD
:1032700009F020E0822F089582E090E00C946439F8
:1032800083E090E00C946439CF9384E090E00E9456
:103290006439C82F82E290E00E9464392C2F30E01C
:1032A000A901582BCA01CF910895CF93C92F682F38
:1032B00084E090E00E9478396C2F82E290E0CF9118
:1032C0000C947839AB01BC018FE090E00C948A3902
:1032D000AB01BC0183E190E00C948A3960E070E0BE
:1032E000CB010C94681969EE7EEF80E090E00E94BB
:1032F000963960E082E090E00E94783960E083E0F7
:1033000090E00E94783910923A0210923B0210929B
:103310003C0210923D0260E084E090E00E94783927
:1033200060E082E290E00E94783960E085E090E021
:103330000E94783960E086E090E00E9478396FEF73
:1033400087E090E00E94783940E050E0BA0188E0E0
:1033500090E00E948A3960E08DE090E00E94783928
:1033600040E050E0BA0188E190E00E948A3960E0D4
:1033700087E190E00E94783940E050E0BA018CE1AA
:1033800090E00E948A3960E070E080E290E00E9464
:10339000963940E050E0BA0188E190E00E948A3915
:1033A0000C940B0C0C947319682F8EE090E00C9425
:1033B00078390E94B2306093D6027093D70280931E
:1033C000D8029093D9026093D2027093D302809373
:1033D000D4029093D502089585B7806885BF85B7DC
:1033E000806885BF089581E008950C94F3190895CD
:1033F0000C94F7190C944E0C0C94F7190C94FC19BE
:103400000C94F7190E94EC198FED92E30E94912E13
:103410000E94001A0C94FE190E94F8190C94F719D6
:103420000E94F61C0E94940E0C942D2A0E949D303E
:103430000E947E1D0E94101A0E945B270E946C242D
:103440000C94FA192F923F924F925F926F927F9253
:103450008F929F92AF92BF92CF92DF92EF92FF92A4
:103460000F931F93CF93DF93CDB7DEB72D970FB692
:10347000F894DEBF0FBECDBF0E94951D282E81118E
:103480000E94D9198AEB92E09D878C8700E010E0BA
:10349000302E802F0E941A1D2B013C01EC85FD85EA
:1034A00081919191A191B191FD87EC8753014201E6
:1034B00088269926AA26BB2681149104A104B1046A
:1034C000B1F40F5F1F4F0630110511F78FEF89839D
:1034D0008A831B820E94A6308160782F9D838C8313
:1034E00049815A816B818D810E94D70E51C0809194
:1034F000DA0281FD0E94261D1B86C12CD12C76018B
:10350000C394D501C4018C219D21AE21BF21892BFB
:103510008A2B8B2B91F10E94F5198823D1F0FB8522
:10352000FE833F824C205D206E207F2081E0452875
:103530004628472809F480E088870E94A6308160E9
:10354000782F9A8789874E815F8168858A850E9456
:10355000D70E000F111F000F111FF801E654FD4F89
:1035600080819181A281B381C826D926EA26FB26D3
:10357000C082D182E282F3820BC08B858F5F8B8702
:10358000CC0CDD1CEE1CFF1C823109F0BACF99CFA8
:1035900081E0211001C080E02D960FB6F894DEBFC7
:1035A0000FBECDBFDF91CF911F910F91FF90EF9094
:1035B000DF90CF90BF90AF909F908F907F906F9053
:1035C0005F904F903F902F9008950E94221A0E9482
:1035D00072250E948D290C94A50ECF93DF930E9433
:1035E000071CEC01811522E59207E8F5811531E50C
:1035F000930708F0B6C0883E910528F5803E9105F6
:1036000008F0E9C0883A910570F4853A910508F010
:103610007AC08130910509F473C008F4D9C00497C9
:1036200008F0D9C0D5C08F3B910508F0D1C0C85A69
:10363000D0E0CC0FDD1FC159DE4F0990D881C02DDD
:10364000CE019464C9C0811540E5940708F069C0B3
:10365000811550E4950708F060C09A9581159F4147
:1036600008F4B9C0B5C0811536E5930728F5811572
:1036700045E5940708F092C0811554E5950708F0D8
:1036800087C0AC0143705527282F26952695C11574
:10369000D34508F06CC081E090E002C0880F991F0C
:1036A0004A95E2F740E2249F90011124EC01C22BDD
:1036B000D32BCE019C6890C081152AE5920780F437
:1036C000811539E5930708F072C0811548E5940724
:1036D00008F47EC0D82FCC27CE01806F906A7CC0C2
:1036E00090568115904208F073C08D2F8F710E9403
:1036F0009B1CDD27D0628F71AE01582BCA016CC0B4
:1037000081E090E069C0C55AD0E0C356DE4F8881A1
:10371000C82FD0E0CE0190645FC0DF70CE01906A08
:103720005BC074E0969587957A95E1F7282F237012
:103730003C2F337081E090E002C0880F991F3A95CA
:10374000E2F79C68AC01522B9A019C2F9F709695D2
:10375000969550E2959FE0011124C9018C2B9D2B79
:103760003BC0D82FCC27CE01816F906A35C081E055
:1037700090E002C0880F991F4A95E2F750E2259F1A
:1037800090011124EC01C22BD32BCE019A6824C0E6
:10379000D82FCC27CE01846F906A1EC00E949B1C3C
:1037A0008F7190E0D82FCC27CE01906215C08F701A
:1037B0000E949B1C94E0D695C7959A95E1F7CF702F
:1037C000D0E0DC2FCC27D0699E01282BC90104C092
:1037D00080E090E001C0CE01DF91CF9108952CE60A
:1037E000829FC0011124FC0122E1729FE00DF11DB6
:1037F0001124E60FF11DEE0FFF1FE158FE4F8591DA
:10380000949108950E94EF1B0E94ED1A089582384A
:10381000910569F1B0F48133910509F46DC048F464
:103820008932910509F463C08A32910509F469C0AF
:1038300008958533910509F455C089339105B9F090
:103840000895833E910569F138F4803E9105B1F009
:10385000823E910509F10895863E9105A9F1873EC2
:103860009105B9F1843E910509F064C023C020910F
:10387000240320FD4FC021FD4DC0089580912403F5
:1038800080FD44C08091250380FF44C080912403C3
:1038900084FD42C083EE4DC08091240382FF38C076
:1038A000F5CF8091240382FD33C08091250380FDF4
:1038B00031C0ECCF8091250381FF32C08091240379
:1038C00084FD2AC087EE35C08091240383FF26C083
:1038D000F5CF8091240383FD21C08091250381FDD4
:1038E0001FC0ECCF8091240385FD1CC01DC08091BA
:1038F000240385FD19C016C08091240386FD16C0DF
:1039000017C08091240386FD13C010C089E311C045
:1039100082EE0FC080EE0DC080E00BC086EE09C0C5
:1039200084EE07C089E205C085E303C08AE201C0D6
:1039300081E390E008959091240392FF0DC0282F19
:103940002871283019F4877F846006C0282F2471DD
:10395000243011F48B7F886093FF0DC0282F2871CD
:10396000283119F4877E846106C0282F2471243100
:1039700011F48B7E88612091250320FF0DC0382F24
:103980003871383019F4877F816006C0382F317163
:10399000313011F48E7F886021FF0DC0282F2871EF
:1039A000283119F4877E816106C0282F21712131C9
:1039B00011F48E7E886194FD877E08950C942B19F6
:1039C0000E94951D8FE39CE90197F1F700C000006C
:1039D0000E94951D80E00E941A1D60FF04C00E9495
:1039E000DE1C0C94F33008950C94E01C0E943119F5
:1039F000811102C00E94D2190E943C198093DA0200
:103A00000E94441990932503809324030E94F41C80
:103A10000E944019682F70E080E090E00E94391306
:103A2000609136027091370280913802909139028C
:103A30000C94711324E0829FC0011124FC01E25C0C
:103A4000FC4F60817181828193810895CF92DF92D2
:103A5000EF92FF920F931F93CF93DF938AE394E04B
:103A60000E9472098EE3E82E83E0F82EC0E0D0E0D9
:103A700095E3C92E94E0D92E0BE214E0DF93CF93A7
:103A8000DF92CF920E940B0A82E394E00E947209B7
:103A9000F70161917191819191917F010E94630E73
:103AA0009F938F937F936F931F930F930E940B0AA3
:103AB00089E294E00E94720921968DB79EB70A961A
:103AC0000FB6F8949EBF0FBE8DBFC630D105B1F6BC
:103AD000DF91CF911F910F91FF90EF90DF90CF90EA
:103AE000089580EA8A95F1F7089508950C94751D5C
:103AF0000C94761D0C94751D0C947A1D0E94B10BCC
:103B0000E6E2F3E0AEE3B3E011921192119211926A
:103B10001D921D921D921D9283E0EE33F807A1F7CE
:103B200086E00E94A81D0C94CA0CCF9386E293E015
:103B30000E94B30BC82F282F46E06EE373E086E2A5
:103B400093E00E94A91D0E94CC0C8C2FCF91089568
:103B50000895FF920F931F93CF93DF93F82ED92FE1
:103B60008B01C42F222349F081E08093DD020E9463
:103B7000A6309093DC028093DB028091DD028823E3
:103B8000F1F08091DB029091DC020E94BE3005973B
:103B9000B0F0EF2DFD2FD80180E090E04C2F50E0E9
:103BA0008417950754F401911191219131910D934E
:103BB0001D932D933D930196F3CF1092DD02DF917B
:103BC000CF911F910F91FF9008950E945B330E9447
:103BD000161A0C9467330E946B330E94E51A0C94FA
:103BE00089330E9444300E9442330E94021A0E948C
:103BF000E51D0E94EB1D0E940C1AFBCFEF92FF9275
:103C00000F931F93CF93DF938B01682F11110AC07D
:103C1000442329F0E82FF0E0EF5DF54F6491762F13
:103C2000862F75C0212F30E0E82FF0E0442321F0EB
:103C3000EF5DF54FE491F0E046E0049FC0011124F0
:103C4000CFEFD0E0BE010E94C6384BEA4603C00168
:103C5000479F900D1124800F911D800F911D982F6B
:103C6000990F890FAE01421B530B4E9FD0014F9FFE
:103C7000B00D5E9FB00D11249B2F189FA001112441
:103C8000452F55278E01041B150B0E9FA0010F9F7A
:103C9000500D1E9F500D11247E01E81AF108E29E7E
:103CA0008001E39E100DF29E100D1124212F332769
:103CB000C21BD30BCE9F9001CF9F300DDE9F300DE6
:103CC000112462307105A9F048F46115710569F09D
:103CD00061307105C9F48B2F752F0DC064307105EB
:103CE00081F058F06630710579F47E2F8B2F932F79
:103CF0000DC0832F7B2F9E2F09C08E2F7B2F952FDA
:103D000005C08E2F732F02C07E2F852F692FDF9164
:103D1000CF911F910F91FF90EF90089541E00E9485
:103D2000FE1D089508958B3170F4262F30E0280F82
:103D3000311D2C3131053CF480930901860F8093AD
:103D40000A0160930B0108950E948E1E0895CF937F
:103D5000DF93762FE901682F842F0E94A41E7983B8
:103D600068838A83DF91CF910895493C08F048EC3D
:103D70000C94A71E80915603282F269530E021151C
:103D8000310519F48170826005C02532310524F0B7
:103D9000817088648093560380915903893C18F0A0
:103DA00088EC80935903089588E090E00C946C3976
:103DB000CF92DF92EF92FF926B017C010E94BA1EBC
:103DC000B701A60188E090E0FF90EF90DF90CF90E0
:103DD0000C948A39E6E5F3E083E0808311828FEF6B
:103DE000828388EC838314826081718182819381D4
:103DF0000C94D81E8091DA0280FF08C089E997E010
:103E00009F938F930E940B0A0F900F908091DA027C
:103E100080FF0FC08091560381701F928F938CE7B3
:103E200097E09F938F930E940B0A0F900F900F9033
:103E30000F908091DA0280FF0FC080915603869523
:103E40001F928F9381E697E09F938F930E940B0AB6
:103E50000F900F900F900F908091DA0280FF0EC0AC
:103E6000809157031F928F9387E497E09F938F93DE
:103E70000E940B0A0F900F900F900F908091DA0222
:103E800080FF0EC0809158031F928F938DE297E0C0
:103E90009F938F930E940B0A0F900F900F900F909B
:103EA0008091DA0280FF0EC0809159031F928F9398
:103EB00083E197E09F938F930E940B0A0F900F90DE
:103EC0000F900F908091DA0280FF0EC080915A030C
:103ED0001F928F9387EF96E09F938F930E940B0A18
:103EE0000F900F900F900F9008958091560380FFD0
:103EF00002C08695089580E0089590915A0393300A
:103F000018F49F5F90935A03882351F060915603F1
:103F10007091570380915803909159030C94D81EC7
:103F2000089581E00C947D1F90915A03992319F014
:103F3000915090935A03882351F0609156037091E9
:103F4000570380915803909159030C94D81E0895FB
:103F500081E00C94941F70E00C94432A6091080156
:103F60008091560380FF0AC08091070123E0829F61
:103F7000C0011124855A9C4F0C94AB1F80910901FC
:103F800090910A01891780F7E82FF0E09F01220F36
:103F9000331FE20FF31FE55AFC4F11821082128289
:103FA0008F5FF0CF9091560390FF16C0909109015A
:103FB00020910A01921770F4E92FF0E0DF01AA0FB7
:103FC000BB1FEA0FFB1FE55AFC4F818360834283CE
:103FD0009F5FF0CF0C94AE1F0895CF93DF9300D076
:103FE0001F92CDB7DEB79091560390FF0AC09E0195
:103FF0002F5F3F4F0E94B51E4B8169818A810E94CD
:10400000D21F0F900F900F90DF91CF910895CF9313
:10401000DF93EC01EC81F0E0EC53F84F4491E6E5DE
:10402000F3E0628181810E94ED1F8C818F5F8C8320
:10403000DF91CF910895CF93DF93EC01E6E5F3E0B4
:10404000438162818C810E94ED1F8C818F5F8C8304
:10405000DF91CF9108950F931F93CF93DF9300D0FB
:104060001F92CDB7DEB78C018091DE0281110AC0AC
:104070009E012F5F3F4F48EC6FEF0E94B51E8A8173
:104080008093DE02F8018481813051F028F0823083
:1040900061F44091DE020AC08091DE0240E007C078
:1040A0006091DE0240E080E003C040E080E060E03C
:1040B0000E94D21FF801848190E0019663E070E0D5
:1040C0000E94DA3884830F900F900F90DF91CF9188
:1040D0001F910F9108954F925F926F927F928F92EE
:1040E0009F92AF92BF92CF92DF92EF92FF920F9387
:1040F0001F93CF93DF9300D01F92CDB7DEB7F82E7A
:10410000B62EE42E622E9091560390FFB4C0E92F94
:10411000E695AE2FB0E0A056BE4F8C918093EA0298
:104120009E7F923061F49E012F5F3F4F8F2D0E9442
:10413000B51E4B8169818A810E94D21F62C0823084
:1041400019F4E09059035DC0863019F4F0905703DC
:1041500058C08930D9F3893109F053C0E9518E2F05
:104160008170782E81E0A72CA826E695F0E0EC532C
:10417000F74FC590D490412CDD249FED892E94E01B
:10418000992E60910B014616D0F5042D10E00C9D80
:10419000C0010D9D900D1C9D900D112470E00E949A
:1041A000C6385F2C711002C0560E01C0561A80919D
:1041B000DA0280FF11C0DF92CF921F92AF921F925E
:1041C0005F921F924F929F928F920E940B0A0FB69E
:1041D000F894DEBF0FBECDBF80910901080F111DFD
:1041E0009801220F331F020F131F9801255A3C4FCD
:1041F0004E2D6B2D852D0E94B51E4394C2CF0E947B
:10420000AE1FF0925703B0925803E0925903662014
:10421000E9F0609156037091570380915803909193
:1042200059030E94D81E8091DA0280FF24C0809139
:1042300059031F928F93809158031F928F938091FF
:1042400057031F928F938AEB94E00CC08091DA029F
:1042500080FF11C01F92EF921F92BF921F92FF9298
:1042600083E994E09F938F930E940B0A0FB6F89412
:10427000DEBF0FBECDBF0F900F900F90DF91CF919B
:104280001F910F91FF90EF90DF90CF90BF90AF9074
:104290009F908F907F906F905F904F900895E6E58C
:1042A000F3E09181282F4381628188E0890F0C948B
:1042B0006B2081E00C944F21E6E5F3E09181282FFB
:1042C0004381628188EF890F0C946B2081E00C940C
:1042D0005C21E6E5F3E0628128E0620F08F46FEF0D
:1042E000282F438181810C946B2081E00C946921FB
:1042F000E6E5F3E0628128E0621B08F460E0282F25
:10430000438181810C946B2081E00C947821E6E557
:10431000F3E0438128E0420F08F44FEF282F628139
:1043200081810C946B2081E00C948721E6E5F3E019
:10433000438128E0421B08F440E0282F62818181FC
:104340000C946B2081E00C94962121E00C946B205E
:1043500020E00C946B20FF920F931F93CF93DF9379
:10436000EC01F12C0FEF10E060910B01F616F0F468
:10437000809109012F2D30E0280F311DC901880FD0
:10438000991F280F391F255A3C4F70E0C8010E9421
:10439000DA38962F8C814091590360915803F99E29
:1043A000800D11240E94B51EF394DECF0E94AE1F33
:1043B0009A818C8190FF02C08F5F01C081508C83F5
:1043C000DF91CF911F910F91FF900895AF92BF920F
:1043D000CF92DF92EF92FF920F931F93CF93DF93D1
:1043E000FC01828180FF02C00FEF01C001E010E0FC
:1043F0004BE1A42E80910B01181708F043C0809167
:104400000901C12ED12CE601C80FD11DCE01880FA4
:10441000991FC80FD91FC55ADC4F198218821A82FA
:1044200034E0E32EF12CB12C8091E0028B0D8C3125
:104430002CF06A2D0E94B838892F05C087FF03C071
:1044400090910B01890F082E000C990BC816D90604
:1044500091F4809159038E9DA0018F9D500D1124E0
:1044600055954795559547959E01609158038091C4
:1044700057030E94B51EB00EF1E0EF1AF108A1F645
:104480001F5FB8CF0E94AE1F8091E002013031F46F
:10449000811102C080910B01815007C090E001960C
:1044A00060910B0170E00E94DA388093E002DF91A6
:1044B000CF911F910F91FF90EF90DF90CF90BF9021
:1044C000AF900895CF938091090190910A018917C7
:1044D00070F4E82FF0E09F01220F331FE20FF31F6B
:1044E000E55AFC4F1182108212828F5FF0CFC0E03C
:1044F00060910B01C617C0F5EC2FF0E070E0CF0122
:104500000E94DA3820910901820F2091DF02022EE9
:10451000000C330B90E0E217F307CCF0209106017A
:10452000022E000C330B2E173F078CF09C01220F3C
:10453000331F820F931F9C01255A3C4F4091590312
:1045400060915803809157030E94B51E0BC0FC0177
:10455000EE0FFF1F8E0F9F1FFC01E55AFC4F1182CB
:1045600010821282CF5FC4CF0E94AE1F209105013E
:104570008091DF02820F8093DF0290910601920FFB
:104580009093060119165CF4082E000C990B4091CB
:104590000B0150E041505109841795071CF02195FB
:1045A00020930501CF9108958F929F92AF92BF9271
:1045B000CF92DF92EF92FF920F931F93CF93DF93EF
:1045C0008C01FC014481C42FD0E09E01DE010E94D9
:1045D00021399B01AC010E9437396B017C01E0E27B
:1045E000F0E0EC1BFD0BA5E5B0E09B01AC010E94E7
:1045F00037394B015C019F01DF010E9419399B0192
:10460000AC010E9442399B01AC012C0D3D1D4E1D99
:104610005F1DC501B4010E94EE38C22FD22F2A328D
:1046200028F4F3E02F9F900111240DC025E530E020
:104630002C1B3109C901880F991F280F391F37FF1B
:1046400002C02F5F3F4F35952795C22FC095F12CA3
:1046500085E5E82EED1A80910B01F816C8F4F1FCFF
:1046600002C08E2D01C08D2F909109012F2D30E0B9
:10467000290F311DA901440F551F240F351F255A3D
:104680003C4F4C2F609158030E94B51EF394E3CF2A
:104690000E94AE1FF8018481811102C091E003C025
:1046A000803219F49FEF9093040190910401890FD7
:1046B000F8018483DF91CF911F910F91FF90EF90CC
:1046C000DF90CF90BF90AF909F908F9008950F9301
:1046D0001F93CF93DF93EC0100E010E080910B017A
:1046E000282F30E00217130724F590910901980153
:1046F000290F311DA901440F551F240F351F255ABD
:104700003C4F869590E04C81081719071CF4442310
:1047100031F002C0411103C04091590301C040E093
:1047200060915803809157030E94B51E0F5F1F4F81
:10473000D5CF0E94AE1F8C8190E0019681709927A1
:104740008C83DF91CF911F910F9108956091560353
:10475000669570E04BE050E08CE091E00E944A39B1
:10476000892B19F481E08093EB020E94A63090938C
:10477000E2028093E1028091DA0280FF08C08AE7BA
:1047800094E09F938F930E940B0A0F900F900895CF
:104790001092EB028091DA0280FF08C081E694E07B
:1047A0009F938F930E940B0A0F900F900895909102
:1047B000560390FF54C09170811102C0926006C0F0
:1047C000853210F0986402C0880F982B909356039E
:1047D0006623B1F06091560370915703809158039E
:1047E000909159030E94D81E8091DA0280FF1BC06D
:1047F0008091560386951F928F938DE396E00BC0B0
:104800008091DA0280FF0FC08091560386951F9237
:104810008F938FE196E09F938F930E940B0A0F90E6
:104820000F900F900F9060915603669570E04BE0EB
:1048300050E08CE091E00E944A39892B19F00E94E7
:10484000C82302C00E94A62381E08093E402409125
:10485000590360915803809157030C94A82108953F
:10486000682F90915603969581E0890F853208F064
:1048700081E00C94D72381E00C943024682F909130
:10488000560396958FEF890F09F484E20C94D72391
:1048900081E00C943E2461E00C94D7238091560370
:1048A0008160809356038091DA0280FF0DC01F92D1
:1048B00081E08F9381EB95E09F938F930E940B0A89
:1048C0000F900F900F900F908091560386950C9447
:1048D0004B2460E00C94D7238091E902811160C0E1
:1048E0008091DA0280FF08C080EE96E09F938F935C
:1048F0000E940B0A0F900F908091DA0280FF08C08F
:104900008AEC96E09F938F930E940B0A0F900F9072
:104910000E943119811110C08091DA0280FF08C015
:1049200082EA96E09F938F930E940B0A0F900F905C
:104930000E94D2190E94EA1E0E94D41E6093560360
:104940007093570380935803909359036E7FC1F47B
:104950008091DA0280FF08C089E596E09F938F93EB
:104960000E940B0A0F900F900E94EA1E0E94D41E14
:1049700060935603709357038093580390935903A1
:104980000E94BA1E0E94FA1E1092EB0280915603FA
:1049900080FF03C086950E94692481E08093E9022C
:1049A0000895809156038160809356038091DA02C6
:1049B00080FF0DC01F9281E08F9388E795E09F9361
:1049C0008F930E940B0A0F900F900F900F90809181
:1049D000560386950C9469241092E8028091E702B0
:1049E00081110E94D1240C94A623809156038E7FBE
:1049F000809356036091560370915703809158033A
:104A0000909159030E94D81E8091DA0280FF0FC056
:104A10008091560381701F928F9380E495E09F935D
:104A20008F930E940B0A0F900F900F900F900E948F
:104A3000C8232FEF80E792E0215080409040E1F7BB
:104A400000C000000C94AE1F8091DA0280FF10C0FD
:104A500080915603809581701F928F9388EE95E028
:104A60009F938F930E940B0A0F900F900F900F90BF
:104A70008091560380FD0C94F5240C944E24809173
:104A800056038E7F809356038091DA0280FF0CC01C
:104A90001F921F9286E095E09F938F930E940B0ACE
:104AA0000F900F900F900F900E94C8232FEF80E778
:104AB00092E0215080409040E1F700C000000C944B
:104AC000AE1F0E94C8238091E80281110AC081E0D4
:104AD0008093E8028091560381708093E7020C94E2
:104AE0003F2508950F931F93CF93DF938091EB029F
:104AF000882309F485C08091EA02E0915603E69587
:104B0000E81BE093E302823049F4F0E0E054F84F10
:104B1000E491CE2FD0E007E010E249C0863049F49E
:104B2000F0E0E354F84FE491CE2FD0E00BE110E237
:104B30003EC0893051F4E695F0E0E654F84FE49138
:104B4000CE2FD0E00BEA11E232C08F3051F4E6955F
:104B5000F0E0E954F84FE491CE2FD0E006EE11E2F8
:104B600026C0853149F4F0E0EC54F84FE491CE2FA3
:104B7000D0E002E612E21BC0883181F0833239F4C2
:104B8000E2EBF7E0C591D4910BE210E210C0843261
:104B900051F4C4EFD1E007E613E209C0C8E2D0E067
:104BA00004ED12E204C0C0EDD7E002E91EE18091FD
:104BB000E402882361F01092E4020E94A6309093F0
:104BC000E2028093E1021092E6021092E5020E9456
:104BD000A630E091E102F091E2028E1B9F0B8F3F25
:104BE0009F4770F4EC0FFD1FF093E202E093E102A7
:104BF00081EE92E0F801DF91CF911F910F9109941E
:104C0000DF91CF911F910F910895882311F0FA0140
:104C100001C0FB010994CF93DF93C82FD62F0E94C8
:104C2000751F8C1740F00E94751F8D1720F4DF91BF
:104C3000CF910C943B248C2FDF91CF910C944B247B
:104C40001F93CF93DF93FB0112811111C3C0EC01BD
:104C50000E9434188272CD3CFCE5DF0709F49AC04B
:104C6000A8F5C73CECE5DE0709F476C0A8F4C43C1F
:104C70009CE5D90709F45FC028F4C33CDC4509F47E
:104C800057C054C0C53C9CE5D90709F459C0C63C7F
:104C9000DC4509F45CC04AC0CA3CFCE5DF0709F406
:104CA0006AC050F4C83CECE5DE0709F45AC0C93CC0
:104CB000DC4509F45BC03AC0CB3C9CE5D90709F45C
:104CC0005FC0CC3CDC4509F460C030C0C23DFCE5AF
:104CD000DF0709F46FC088F4CF3C9CE5D90709F4DD
:104CE00060C008F45CC0C03DFCE5DF0709F45CC0AF
:104CF000C13DDC4509F45BC019C0C53D9CE5D90741
:104D000009F460C050F4C33DFCE5DF0709F455C069
:104D1000C43DDC4509F454C009C0C63D9CE5D90733
:104D200009F455C0CE35DD4509F454C011E052C038
:104D30000E9424254FC048E454E26BE374E204C0AF
:104D40004BE354E268E474E20E94052643C046E661
:104D500051E269E571E2F8CF49E551E266E671E2B8
:104D6000F3CF44E851E265E771E2EECF45E751E267
:104D700064E871E2E9CF42EA51E263E971E2E4CF2B
:104D800043E951E262EA71E2DFCF48EA5FE161E9BB
:104D90007FE1DACF41E95FE168EA7FE1D5CF81E0E9
:104DA00017C065E082E010C068E086E00DC06EE0EC
:104DB00089E00AC064E18FE007C067E185E104C0D3
:104DC00088E106C062E289E10E940B2603C083E20B
:104DD0000E944B24812FDF91CF911F91089586E08F
:104DE00090E00C946439682F86E090E00C94783958
:104DF0008091AC03847089618093AC030C94F3269A
:104E00008091AC0386958695869508958091AC0334
:104E100081FD13C082608093AC030E94F3268091D1
:104E2000DA0280FF08C086EE98E09F938F930E947D
:104E30000B0A0F900F900C948E2908958091AC036B
:104E400081FF13C08D7F8093AC030E94F326809175
:104E5000DA0280FF08C089EC98E09F938F930E944C
:104E60000B0A0F900F900C949A290895CF93C0913C
:104E7000AC03C695C1708091DA0280FF0CC01F920E
:104E8000CF9382E099E09F938F930E940B0A0F903B
:104E90000F900F900F90CC2319F0CF910C941E27F8
:104EA000CF910C9406278091AC038695817008956C
:104EB0008091170108950E943119811104C00E9448
:104EC000D2190E94F8260E94EF268093AC03282F67
:104ED00026952695269530E02430310524F08770FC
:104EE00088618093AC038091AC0380FF04C08695F9
:104EF0008695869501C080E00C945B292091AC03D7
:104F0000822F869586958695482F50E0433051052F
:104F100054F48F5F982F990F990F990F822F8770F4
:104F2000892B8093AC038091AC0381608093AC03A8
:104F30000E94F3268091DA0280FF11C08091AC03B9
:104F40008695869586951F928F9389E899E09F9321
:104F50008F930E940B0A0F900F900F900F908091EB
:104F6000AC038695869586950C945B298091AC035D
:104F7000982F969596959695A1F0915E990F990F19
:104F8000990F8770892B8093AC03887F91E009F497
:104F900090E08091AC0390FB80F98093AC030E9479
:104FA000F3268091DA0280FF11C08091AC038695D0
:104FB000869586951F928F9381E799E09F938F93B3
:104FC0000E940B0A0F900F900F900F908091AC03EE
:104FD0008695869586950C945B298091AC0380FD1F
:104FE0001FC081608093AC03813019F489E0809305
:104FF000AC038091AC030E94F3268091DA0280FF1B
:1050000008C089E499E09F938F930E940B0A0F9048
:105010000F908091AC038695869586950C945B29BC
:1050200008958091AC0380FF14C08E7F8093AC0301
:105030000E94F3268091DA0280FF08C086E399E09F
:105040009F938F930E940B0A0F900F9080E00C9417
:105050005B290895CF93C091AC03C1708091DA02AF
:1050600080FF0CC01F92CF938BE599E09F938F93A5
:105070000E940B0A0F900F900F900F90CC2319F005
:10508000CF910C941128CF910C94ED279091AC0303
:10509000892F8695869586958F5F8F71977084305E
:1050A00038F4880F880F880F892B8093AC0302C0D7
:1050B0009093AC038091AC03887F91E009F490E079
:1050C0008091AC0390FB80F98093AC030E94F3269F
:1050D0008091DA0280FF11C08091AC03869586959D
:1050E00086951F928F9382E299E09F938F930E94FF
:1050F0000B0A0F900F900F900F908091AC03869544
:10510000869586950C945B29843008F083E0909115
:10511000AC039770282F220F220F220F922B90930F
:10512000AC03987F21E009F420E09091AC0320FBD0
:1051300090F99093AC030C945B290E948428809191
:10514000AC030C94F326FC01DB0112968C918823AE
:10515000F9F0EC5BFC45E730F105D8F4E85AFF4F75
:105160000C94103983E001C080E00E949D2880E00B
:1051700008950E94B627FBCF0E947E27F8CF0E9499
:105180002A28F5CF0E944628F2CF0E943627EFCF7B
:1051900081E00895279A2F9808952F9808958F9267
:1051A0009F92AF92BF92CF92DF92EF92FF920F93B6
:1051B0001F93CF93DF938C0180918600909187009D
:1051C0006CE070E00E94C6386017710730F0C801CB
:1051D00069E070E00E94C63860C0809186009091BE
:1051E0008700E0908600F0908700E0918600F091C3
:1051F0008700C6E0D0E0BE010E94C63820E030E063
:10520000060F171F211D311D4801590185E0880C2B
:10521000991CAA1CBB1C8A95D1F7C701BE010E942C
:10522000C6386F01E12CF12CA7019601260F371F1C
:10523000411D511DC501B4010E94EE3869017A017A
:10524000E0918600F0918700CA01B9010E949C3864
:105250009B01AC01DF010E9437399B01AC01C70102
:10526000B6010E949C38DC01CB012FE0B695A795D2
:10527000979587952A95D1F7009186001091870020
:1052800020E030E0081719072A073B0728F460914F
:10529000860070918700CB01BC01CB01DF91CF91DB
:1052A0001F910F91FF90EF90DF90CF90BF90AF9044
:1052B0009F908F900895CF93C82F843050F4811120
:1052C00009C080918000877F809380000E94CD2854
:1052D00006C0C3E080918000886080938000A09128
:1052E0008600B09187002C2F30E00E94213923E006
:1052F00030E040E050E00E94EE38B42FA32F922F10
:105300008827892F9A2FAB2FBB270E94CF289093F5
:105310008D0080938C00CF91089508951092ED0236
:105320001092EC021092EE02EFE6F0E080818160D4
:1053300080830895EFE6F0E080818E7F80830E9475
:1053400000270C945B291F920F920FB60F92112425
:105350000BB60F920F931F932F933F934F935F932F
:105360006F937F938F939F93AF93BF93CF93EF935D
:10537000FF938091180191E0980F823019F090937B
:10538000180155C081E0809318010E945827C82F4A
:105390000091EC021091ED020F5F1F4F0E94582701
:1053A00028E7829FB0011124C8010E94C63890935B
:1053B000ED028093EC0228E7C29FB0011124660F32
:1053C000672F661F770B71950E94C6386F778091A3
:1053D000EE02823019F4603451F404C0813039F4A3
:1053E0006F3729F480916F008E7F80936F00E62FD6
:1053F000F0E0EF55F64FC4910091860010918700C0
:105400000E940027282FC09FC001C19F900D11242A
:105410006DEF72E00E94C638269FC001279F900D55
:1054200011240E94CF2890938D0080938C00FF91CF
:10543000EF91CF91BF91AF919F918F917F916F919C
:105440005F914F913F912F911F910F910F900BBE44
:105450000F900FBE0F901F9018950E94CA288AE0E7
:105460008093800089E1809381008FEF9FEF90937C
:105470008700809386000E945B270E94532781113A
:105480000C948E290895209A25B12E7F35B1316074
:105490004FB7F894FC01CB01880F991F680F791F53
:1054A0006E0F7F1FE617F70789F0819198E035B9F5
:1054B000000000C087FF25B9880F000000C000C0B1
:1054C00000C025B900C09A9591F7ECCF4FBF8FE58A
:1054D00094E00197F1F700C000000895CF93DF93A7
:1054E000EC01FB018281882309F43CC1C430FDE555
:1054F000DF0760F4CB3F9CE5D90788F49E0122507A
:105500003C452431310508F02EC109C0C236EDE515
:10551000DE0729F0C63AFDE5DF0709F024C10E9445
:1055200044199093250380932403C1318CE5D80757
:1055300009F4C6C008F042C0C930ECE5DE0709F442
:105540009BC000F5C5308CE5D80709F485C078F418
:10555000C330ECE5DE0709F478C008F07AC0C23049
:10556000DC4509F0F5C0809124038160EFC0C730AD
:105570009CE5D90709F478C008F07AC0809124032B
:105580008061E4C0CD30FCE5DF0709F487C058F442
:10559000CB309CE5D90709F479C008F07BC0809135
:1055A000240388606FC0CF30FCE5DF0709F480C0BA
:1055B00008F082C080912403877FC8C0CE3F9CE55D
:1055C000D90709F471C000F5C531FCE5DF0709F41E
:1055D00085C068F4C3319CE5D90709F475C008F0AB
:1055E00095C00E94E112809124038F77AFC0CC3F19
:1055F000FCE5DF07A9F108F054C0CB3FDC4509F01A
:10560000A7C08091250340C0C230EDE5DE0709F454
:1056100089C058F4C1158DE5D80709F45AC008F0BF
:1056200069C08091250382602FC0C236EDE5DE0798
:1056300009F47CC0C63AFDE5DF0709F481C0C33038
:10564000DD4509F085C080E06EC080912403826052
:105650007DC08091240316C080912403886076C0A9
:105660008091250382604FC08091240380626EC0C8
:105670008091240380646AC00E94E1128091240317
:10568000806864C0846062C081603DC080912403F2
:105690008E7F5CC0809124038D7F58C0809124034D
:1056A00016C08091250318C0809125038D7F2BC0E3
:1056B000809124038F7E4AC0809124038F7D46C051
:1056C000809124038F7B42C080912403877F8B7F4E
:1056D0003DC0809125038D7F8E7F15C0809124036E
:1056E00082FB222720F991E0922790FB82F990FB20
:1056F00083F92CC080912503982F909591708E7F0F
:10570000892B90FB81F98093250322C00E94E1122E
:105710008091240387FB222720F991E0922790FBB8
:1057200087F914C081E00E94D41912C0809124032B
:1057300084FB222720F991E0922790FB84F906C090
:1057400080912403982F909590FB80F980932403F7
:1057500080912403909125030E9455190E94E11223
:1057600080E001C081E0DF91CF910895CF93C82FF1
:105770001F928F9387E29BE09F938F930E940B0A67
:1057800081E090E0A0E0B0E0BC01CD0104C0660F74
:10579000771F881F991FCA95D2F70E9439130F905F
:1057A0000F900F900F90CF910C94E112DF92EF9237
:1057B000FF920F931F93CF93DF93482F50E0FA018E
:1057C0003597EF33F10508F05BC1E15AFF4F0C94B8
:1057D00010390E9440191F928F938EE99FE09F938A
:1057E0008F930E940B0A0E943C1983FB992790F922
:1057F0001F929F9382FB992790F91F929F9381FBA1
:10580000992790F91F929F93982F91701F929F93C1
:105810001F928F9385E59FE09F938F930E940B0AC1
:105820000E94441987FB222720F91F922F9386FBA1
:10583000222720F91F922F9385FB222720F91F9200
:105840002F9384FB222720F91F922F9383FB22277B
:1058500020F91F922F9382FB222720F91F922F936A
:1058600091FB222720F91F922F93292F21701F923D
:105870002F9381FB222720F91F922F93282F21702D
:105880001F922F939F938F9380E79EE09F938F9318
:105890000E940B0A8DB79EB788960FB6F8949EBFEC
:1058A0000FBE8DBF0E94EF26982F969596959695E0
:1058B0001F929F93982F91701F929F931F928F9387
:1058C0008DE39EE09F938F930E940B0A8DB79EB746
:1058D00008960FB6F8949EBF0FBE8DBF06C08EE52A
:1058E00090E10E9472090E94D219C1E0CEC08BE8FB
:1058F0009CE074C08091DA02817F8E7F8093DA020F
:1059000080E79CE00E9472098AE590E10E9472099A
:1059100081E08093EF02E9CF8EE390E10E9472096B
:105920000E94CF0CE2CF8091DA02C82FC095C170DF
:10593000C0FB80F98093DA02CC2319F082E390E176
:1059400091C085E290E10E9472098091DA02897F1C
:10595000877F8093DA02C9CF9091DA0291FBCC273E
:10596000C0F981E0C827892FC0FB81F98093DA0252
:10597000CC2319F088E190E127C08AE090E12EC0A5
:105980009091DA0292FBCC27C0F981E0C827892FD9
:10599000C0FB82F98093DA02CC2319F08BEF9FE0F1
:1059A00013C08BEE9FE01AC09091DA0293FBCC27D4
:1059B000C0F981E0C827892FC0FB83F98093DA0200
:1059C000CC2351F08FED9FE00E9472098091DA02A2
:1059D00081608093DA0259C082ED9FE00E947209D3
:1059E00084CF80EB9BE0FACF0E94B230062FF72ED7
:1059F000E82ED92EC0912403C7FBCC27C0F9109103
:105A00002303D09125010E949B2EDF92EF92FF92FB
:105A10000F931F92CF931F921F931F92DF931F929A
:105A20008F938CE29BE09F938F930E940B0A8DB71C
:105A30009EB70E960FB6F8949EBF0FBE8DBF55CF82
:105A40000E94E1129091240397FBCC27C0F981E0DA
:105A5000C827892FC0FB87F980932403CC2329F022
:105A600088EC9FE00E94720910C08DEB9FE0B6CFDA
:105A7000895303C08D5101C080E00E94B62B35CF01
:105A80008BEB9FE00E947209C0E08C2FDF91CF91D9
:105A90001F910F91FF90EF90DF90089580E008959F
:105AA0000C944E2DCF93C82F8091EF02882319F0CC
:105AB000813031F038C00E9434188232B1F504C010
:105AC0000E943418823261F48C2F0E94502D811173
:105AD00004C08C2F0E94D62B24C081E090E021C00E
:105AE0008C2F0E944E2D81111BC0C43189F018F4F7
:105AF000CB3029F010C0C93259F0C83361F480E7C7
:105B00009CE00E94720983E29BE00E94720908C037
:105B10001092EF020CC081E29BE00E94720907C064
:105B200081E0817006C01092EF0280E002C080E048
:105B3000F8CFCF910895CF93DF9386319C4541F5FF
:105B4000EB010E943418982F8A8120910201309134
:105B50000301882379F09A7A81E009F480E0809348
:105B6000F002911102C069E201C065E3C9010E941F
:105B7000E02F0AC08091F002811102C069E201C0E9
:105B800065E3C9010E94EB2F0E94761880E001C0F6
:105B900081E0DF91CF9108950F931F93CF93DF930F
:105BA000C42FD22FFC0182818823C9F04093F302D5
:105BB0000E94A6309093F2028093F10280E28C0F53
:105BC000883008F057C0C77081E001C0880FCA95BF
:105BD000EAF7DF91CF911F910F910C944D108091B6
:105BE000F302481330C08091F1029091F2020E94BA
:105BF000BE30883C910538F510E21D0FCD17B9F085
:105C000080E28C0F883040F4C77081E001C0880FBB
:105C1000CA95EAF70E945410183028F581E09D2FAC
:105C2000977001C0880F9A95EAF70E944D10802F57
:105C30000E9444101830F0F4D77081E001C0880F42
:105C4000DA95EAF70AC080E28C0F883098F4C770C2
:105C500081E001C0880FCA95EAF7DF91CF911F91CB
:105C60000F910C945410802FDF91CF911F910F91C1
:105C70000C944410DF91CF911F910F9108950F93D1
:105C80009C01CB01243F4CE5340731F188F4293DD8
:105C9000FCE53F07D9F02A3D4CE5340779F1283D72
:105CA0003C45A9F506E221EE41EE68ED7CE52BC00E
:105CB000263FFCE53F07E1F0A8F0273F3C4539F5DA
:105CC00007E225EE46EE67EF7CE51DC007E225EE14
:105CD00045EE69ED7CE517C006E221EE40EE64EF8B
:105CE0007CE511C007E225EE44EE65EF7CE50BC0D4
:105CF00006E221EE42EE66EF7CE505C008E221E017
:105D000045EE6AED7CE50E94CC2D80E008C0FC01E8
:105D10008281882319F01092F30201C081E00F9173
:105D200008959093D5018093D40108959093F9023A
:105D30008093F8020895E091F802F091F90230970B
:105D400021F00190F081E02D099480E00895EF9218
:105D5000FF921F93CF93DF93FC01A091F802B091C3
:105D6000F902109709F442C080912501882341F07F
:105D70008091240387FF04C08081818386E0808333
:105D8000EF011296ED91FC911397CE010995809148
:105D9000DA0282FF2BC080FF04C087E790E10E94F7
:105DA000720918E081E7E82E80E1F82E8091DA028E
:105DB00080FF0BC088811F928F93FF92EF920E9409
:105DC0000B0A0F900F900F900F9011502196111108
:105DD000EDCF8091DA0280FF09C08FE690E1DF917C
:105DE000CF911F91FF90EF900C947209DF91CF91AA
:105DF0001F91FF90EF9008952091F6023091F702E5
:105E00002817390771F09093F7028093F602E0911A
:105E1000F802F091F902309721F00680F781E02D29
:105E2000099408952091F4023091F502281739075A
:105E300071F09093F5028093F402E091F802F091F2
:105E4000F902309721F00084F185E02D099408953E
:105E5000FC01329680912501882331F08091240342
:105E600087FF02C09EE101C096E080E0915028F0DB
:105E700021912223D9F38F5FF9CF0895662351F141
:105E8000209125012223E9F02091240327FF19C046
:105E9000462F4695469546954E31E0F4677021E0D1
:105EA00030E002C0220F331F6A95E2F7FC01E40FD5
:105EB000F11D828190E02823392381E0232B69F4AE
:105EC00009C0FC01329608962191621729F0E81763
:105ED000F907D1F780E0089581E008959C01FC0165
:105EE00032969FEF80E04191461789F09F3F19F469
:105EF000411101C0982F8F5F8630A9F79F3F39F07D
:105F0000F901E90FF11D97FDFA956283089508954F
:105F10009C012A5F3F4FFC014281461301C012825F
:105F2000019682179307B9F70895262F269526958F
:105F300026952E3170F4FC01E20FF11D677021E00F
:105F400030E001C0220F6A95EAF78281282B228374
:105F500008958091DA0280FF0CC01F926F9387EA48
:105F600090E19F938F930E940B0A0F900F900F90D8
:105F70000F900895262F2695269526952E3178F494
:105F8000FC01E20FF11D677021E030E001C0220F3B
:105F90006A95EAF7209582812823228308958091CB
:105FA000DA0280FF0CC01F926F9389E890E19F9303
:105FB0008F930E940B0A0F900F900F900F900895EF
:105FC00020912501222329F02091240327FD0C9400
:105FD000952F0C946E2F20912501222329F02091DA
:105FE000240327FD0C94BA2F0C94882F20912501AF
:105FF000FC013296222331F08091240387FF02C0F6
:106000008EE101C086E0DF011D928A95E9F70895CF
:1060100008950C94083083E08093FA020C940930C0
:10602000811102C081E001C082E08093FA020C94E9
:1060300009300C94103081E08093FA020C940930FE
:106040000C941B3008950C9422300C9423300C9443
:1060500022300C9422300C942230CF930E942930AD
:106060000E94951D0E942730C0E08C2F0E941A1DAF
:10607000672B682B692B29F4CF5FC630B1F780E01E
:1060800001C081E0CF91089508951F920F920FB63D
:106090000F9211248F939F93AF93BF938091FB0234
:1060A000811113C08091AD039091AE03A091AF0315
:1060B000B091B0034196A11DB11D8093AD039093A3
:1060C000AE03A093AF03B093B003BF91AF919F9184
:1060D0008F910F900FBE0F901F9018958091B50370
:1060E000843031F10E94570D1092FB0220E488E1C8
:1060F00090E00FB6F894A895809360000FBE2093AF
:10610000600083B7817F846083BF83B7816083BF72
:106110007894889583B78E7F83BF0FB6F894A8953F
:1061200080916000886180936000109260000FBED3
:1061300008950E94E1120C94600D82E084BD93E00A
:1061400095BD9AEF97BD80936E0008952FB7F89490
:106150008091AD039091AE03A091AF03B091B003D5
:106160002FBF08952FB7F8946091AD037091AE03DF
:106170008091AF039091B0032FBF08959C014FB75A
:10618000F8948091AD039091AE03A091AF03B091CC
:10619000B0034FBF821B930B089578941F920F9208
:1061A0000FB60F9211248F939F93AF93BF9380915B
:1061B000AD039091AE03A091AF03B091B0030196EF
:1061C000A11DB11D8093AD039093AE03A093AF03C7
:1061D000B093B003BF91AF919F918F910F900FBE7D
:1061E0000F901F90189581E08093E00080E28093EB
:1061F000D8001092C9008FE19EE40197F1F700C02A
:10620000000087E090EBDC018093BE039093BF0316
:10621000A093C003B093C1039CE088E10FB6F8944B
:10622000A895809360000FBE90936000FFCF80918F
:10623000220308950895CF93DF932091250122230F
:1062400039F02091240327FF03C060E222E002C05E
:1062500068E021E02093E9002FEF3091E800215021
:1062600035FD06C035ED3A95F1F700002111F5CF67
:106270002091E80025FF1DC0EC01809125018111CE
:1062800005C040E050E068E070E003C070E040E02E
:1062900050E0CE010E94F8338091E8008E77809321
:1062A000E80080E2FE01A2E0B3E001900D928A9541
:1062B000E1F7DF91CF9108958093FE027093000380
:1062C0006093FF028091B503843001F582E08093F2
:1062D000E9008FEF9091E800815095FD06C095EDA3
:1062E0009A95F1F700008111F5CF8091E80085FFC4
:1062F0000DC040E050E063E070E08EEF92E00E945D
:10630000F8338091E8008E778093E8000895BC010F
:1063100084E00C945C31BC0183E00C945C31089502
:1063200089ED90E10E9472098091B403811109C046
:106330000E9485350E94E7358091E2008460809359
:10634000E200089585ED90E10E9472091092B40375
:10635000089581ED90E10E9472090C9420308DEC3B
:1063600090E10E9472096091B10381E0611101C066
:1063700080E00C940B3089EC90E10E9472099091BE
:10638000B50381E0943009F080E06091B1030C9492
:1063900010302091FD022F5F822F62E30E94AC3803
:1063A000992319F02093FD0208951092FD02809127
:1063B0000103882371F18091B503843041F5809108
:1063C000E9008F702091EC00922F917020FD90E8F1
:1063D000892B93E09093E9009091EB0090FF14C01B
:1063E0009091EE0097FF10C09091E80095FF03C0D8
:1063F0001092F100F9CF9091E80090FF05C09091C4
:10640000E8009E779093E8008F708093E9001092E7
:106410000103089542E061EC81E00E94FE3442E213
:1064200061EC82E00E94FE3442E261EC83E00E9473
:10643000FE349091B50381E0943009F080E06091E2
:10644000B1030C9419308091B703833009F45FC015
:1064500030F4813071F0823009F498C008958A30A8
:1064600009F484C08B3009F46AC0893009F0A6C0F1
:1064700020C08091B603813A09F0A0C08091E80065
:10648000877F8093E8008091BA039091BB03892BAA
:1064900021F460E282E093E003C060E080E090E0FD
:1064A00070E00E9443348091E8008B778093E8008D
:1064B00008958091B603813209F080C08091BA03BB
:1064C0009091BB03029708F079C08091E800877F24
:1064D0008093E8008091E80082FD05C08091B503BB
:1064E0008111F8CF6BC08091F2009091F300029778
:1064F00031F48091F100813011F0863021F48091E7
:10650000F100809322038091E8008B7753C0809143
:10651000B603813A09F052C08091BA039091BB034F
:10652000892B09F04BC08091E800877F8093E800B9
:106530008091E80080FFFCCF8091250136C08091DA
:10654000B6038132D9F58091BA039091BB03892BB0
:10655000A9F58091E800877F8093E8000E94333599
:106560008091B803809325010C94E1128091B603C9
:10657000813221F58091E800877F8093E8000E94B6
:1065800033358091B9038093230308958091B60336
:10659000813AA1F48091E800877F8093E8008091A0
:1065A000E80080FFFCCF809123038093F10080916D
:1065B000E8008E778093E8000C94333508959FB7F8
:1065C000F894109201039FBF9091B503943009F0A5
:1065D00057C09091E9009F703091EC00232F2170FB
:1065E00030FD20E8922B23E02093E9002091EB007E
:1065F00020FF43C02091EE0027FF3FC02091FC0206
:10660000222321F02091E80025FF37C01092FC02E0
:1066100026E03091E80035FD15C03091B5033430E7
:1066200061F53091EB0035FD28C0215021F481E067
:106630008093FC0222C0EFE9FFE03197F1F700C040
:106640000000E7CF8093F1008091E80085FD0AC04B
:106650008091E80080FFFCCF8091E8008E778093E6
:10666000E80006C08FB7F89421E0209301038FBFA4
:106670009F709093E90080E008959F709093E900E7
:106680008FEF089584B7877F84BF0FB6F894A895DD
:1066900080916000886180936000109260000FBE5E
:1066A00090E080E80FB6F8948093610090936100C9
:1066B0000FBE0C941B300E9485350E94E735E2EE38
:1066C000F0E080818460808378940C94813889E143
:1066D00091E00C94962E8091B5038530C9F485EC39
:1066E00090E10E9472098091B503853079F40E948F
:1066F0006E308091B3038823B1F30E942D3088233C
:1067000091F30E94E2330E94E112EDCF0C94993094
:10671000089508950C948C33292F332723303105A5
:10672000C9F060F42130310581F02230310509F0E3
:1067300041C08BE590E027E131E140C021323105D5
:10674000E1F02232310531F135C082E190E022E7FB
:1067500031E134C099278130910549F028F0029742
:1067600049F5EDEDF0E105C0E3E1F1E102C0E9EE4C
:10677000F0E1849190E09F0121C063307105D0F475
:10678000660F771FFB01E253FE4F2081318189E0C4
:1067900090E014C06330710568F4FB01EE0FFF1F39
:1067A000E853FE4F20813181FB01EB53FE4F808186
:1067B00090E004C080E090E020E030E0FA01318316
:1067C0002083089584E189BD86E189BD09B400FE76
:1067D000FDCF8091D8008F7D8093D8008091E0001C
:1067E00082608093E0008091E00081FDFCCF0895FD
:1067F000CF92DF92EF92FF920F931F93CF93DF938D
:10680000EC018B017A010E945235811133C0E114F1
:10681000F10439F0F70180819181081B190BC80F31
:10682000D91FC12CD12C0115110519F18091E80057
:1068300085FD16C08091E8008E778093E800E11412
:10684000F10449F0F70180819181C80ED91ED182EF
:10685000C08285E00FC00E945235882321F30AC010
:1068600089918093F10001501109FFEFCF1ADF0ADF
:10687000DACF80E0DF91CF911F910F91FF90EF90E1
:10688000DF90CF9008952091BC033091BD0326176F
:10689000370748F06115710539F42091E8002E772B
:1068A0002093E80001C0B901FC0120E061157105E9
:1068B00069F18091B5038823E1F18530E1F18091A0
:1068C000E80083FD3AC08091E80082FD2CC08091F1
:1068D000E80080FFEBCF8091F2009091F30061150A
:1068E000710551F08830910538F421912093F10021
:1068F000615071090196F3CF21E0089709F020E07B
:106900008091E8008E778093E800D0CF2111D1CF1D
:106910000AC08091B503882361F0853061F08091D1
:10692000E80083FD0AC08091E80082FFF2CF80E09A
:10693000089582E0089583E0089581E0089520910C
:10694000BC033091BD032617370748F06115710568
:1069500039F42091E8002E772093E80001C0B901B6
:10696000FC0120E06115710581F18091B503882358
:1069700009F43EC0853009F43DC08091E80083FDF4
:106980003BC08091E80082FD2DC08091E80080FF2F
:10699000E9CF8091F2009091F3006115710559F0F3
:1069A0008830910540F424912093F1003196615094
:1069B00071090196F2CF21E0089709F020E080915B
:1069C000E8008E778093E800CDCF2111CECF0AC0AA
:1069D0008091B503882361F0853061F08091E800F3
:1069E00083FD0AC08091E80082FFF2CF80E0089525
:1069F00082E0089583E0089581E00895982F97300C
:106A000068F59093E900981739F07091EC002091A7
:106A1000ED005091F00003C0242F762F50E021FDAF
:106A200002C09F5FECCF3091EB003E7F3093EB00D4
:106A30003091ED003D7F3093ED003091EB003160FF
:106A40003093EB007093EC002093ED005093F00036
:106A50002091EE0027FDE5CF80E008958F708093B0
:106A6000E90081E008958091B60387FF11C080910D
:106A7000E80082FD05C08091B5038111F8CF11C0F7
:106A80008091E8008B770BC08091B503882349F093
:106A90008091E80080FFF8CF8091E8008E778093A6
:106AA000E80008952091E4003091E50095E64091DA
:106AB000EC00842F817040FF23C08091E80080FDAE
:106AC0001DC08091B503882399F0853099F080919D
:106AD000EB0085FD11C04091E4005091E5002417C2
:106AE000350729F3915011F09A01E1CF84E0089520
:106AF00082E0089583E0089581E0089580E008959C
:106B00004091E80042FFDDCF08950E94F6350E94D3
:106B1000FE35E0EEF0E0808181608083E8EDF0E01A
:106B200080818F77808319BCA7EDB0E08C918E7F38
:106B30008C9380818F7E80831092B40308950F938D
:106B40001F93CF93DF930E94F6350E94FE35C8ED68
:106B5000D0E088818F778883888180688883888166
:106B60008F7D8883E7EDF0E080818068808319BCA9
:106B70001092B5031092B1031092B3031092B203B6
:106B800000EE10E0F80180818B7F80838881816036
:106B9000888342E060E080E00E94FE34E1EEF0E0B5
:106BA00080818E7F8083E2EEF0E08081816080834F
:106BB000808188608083F80180818E7F80838881D6
:106BC00080618883DF91CF911F910F910895E8ED47
:106BD000F0E080818F7E8083E7EDF0E0808181604E
:106BE000808381E08093B4030C949F35E8EDF0E05E
:106BF00080818C7F80831092E20008951092DA00E9
:106C00001092E10008951F920F920FB60F92112477
:106C10000BB60F922F933F934F935F936F937F9396
:106C20008F939F93AF93BF93EF93FF938091E10076
:106C300082FF0BC08091E20082FF07C08091E100DB
:106C40008B7F8093E1000E94C9318091DA0080FF40
:106C50001FC08091D80080FF1BC08091DA008E7F1A
:106C60008093DA008091D90080FF0DC084E189BD56
:106C700086E189BD09B400FEFDCF81E08093B503B4
:106C80000E94903105C019BC1092B5030E94A23138
:106C90008091E10080FF19C08091E20080FF15C063
:106CA0008091E2008E7F8093E2008091E20080611B
:106CB0008093E2008091D80080628093D80019BC54
:106CC00085E08093B5030E94AF318091E10084FF9D
:106CD00030C08091E20084FF2CC084E189BD86E150
:106CE00089BD09B400FEFDCF8091D8008F7D8093CF
:106CF000D8008091E1008F7E8093E1008091E200D6
:106D00008F7E8093E2008091E20081608093E200B8
:106D10008091B103882311F084E007C08091E300E3
:106D200087FD02C081E001C083E08093B5030E942B
:106D3000BB318091E10083FF29C08091E20083FF95
:106D400025C08091E100877F8093E10082E08093FD
:106D5000B5031092B1038091E1008E7F8093E10032
:106D60008091E2008E7F8093E2008091E20080615A
:106D70008093E20042E060E080E00E94FE34809177
:106D8000F00088608093F0000E94A931FF91EF919C
:106D9000BF91AF919F918F917F916F915F914F9133
:106DA0003F912F910F900BBE0F900FBE0F901F9031
:106DB00018951F920F920FB60F9211240BB60F92D7
:106DC0002F933F934F935F936F937F938F939F93F3
:106DD000AF93BF93CF93DF93EF93FF93C091E900FD
:106DE000CF708091EC00D82FD17080FDD0E8109248
:106DF000E9008091F000877F8093F00078940E94F2
:106E000021371092E9008091F00088608093F000B3
:106E1000CD2BCF70C093E900FF91EF91DF91CF911F
:106E2000BF91AF919F918F917F916F915F914F91A2
:106E30003F912F910F900BBE0F900FBE0F901F90A0
:106E400018951F93CF93DF93CDB7DEB7AA970FB6F0
:106E5000F894DEBF0FBECDBFE6EBF3E08091F1000A
:106E6000819323E0EE3BF207C9F70E942332809121
:106E7000E80083FF2EC18091B6039091B703492F9C
:106E800050E04A30510508F024C1FA01E256FF4FA4
:106E90000C941039803821F0823809F01AC108C0EA
:106EA0008091B2039091B303992389F082600FC05F
:106EB0008091BA038F70873008F00BC18093E9008E
:106EC0008091EB0085FB882780F91092E900909172
:106ED000E800977F9093E8008093F1001092F10012
:106EE000D1C0282F2D7F09F0F4C0882319F08230FB
:106EF00061F0EFC08091B803813009F0EAC09330AF
:106F000009F080E08093B3032EC08091B803811113
:106F10002AC08091BA038F702FEF280F263008F017
:106F2000D8C08093E9002091EB0020FF1CC0933073
:106F300021F48091EB00806214C09091EB0090618D
:106F40009093EB0021E030E0A90102C0440F551FEF
:106F50008A95E2F74093EA001092EA008091EB00F4
:106F600088608093EB001092E9008091E800877FB1
:106F70008093E8000E943335ACC08111AAC0109103
:106F8000B8031F778091E3008078812B8093E30022
:106F90008091E800877F8093E8000E9433358091DC
:106FA000E80080FFFCCF8091E30080688093E300DD
:106FB000111102C082E001C083E08093B50389C053
:106FC0008058823008F085C08091B8039091B90351
:106FD0008C3D53E0950779F583E08A838AE28983C3
:106FE0004FB7F894DE01139620E03EE051E2E32F24
:106FF000F0E050935700E49120FF03C0E295EF705A
:107000003F5FEF708E2F90E0EA3010F0C79601C01E
:10701000C0968D939D932F5F243149F74FBF809188
:10702000E800877F8093E8006AE270E0CE01019675
:107030000E94433416C06091BA037091BB03AE0145
:107040004F5F5F4F0E948A33BC01892B09F441C016
:107050009091E800977F9093E80089819A810E943F
:107060009F348091E8008B778093E80032C08038AD
:1070700081F58091E800877F8093E8008091B103DB
:107080008093F1008091E8008E7772CF811121C04A
:107090008091B8039091B90399270297D4F4809115
:1070A000E800877F8093E8008091B8038093B10364
:1070B0000E9433358091B103811106C08091E300B5
:1070C00087FD02C081E001C084E08093B5030E9487
:1070D0000A328091E80083FF0AC08091E800877F30
:1070E0008093E8008091EB0080628093EB00AA9689
:1070F0000FB6F894DEBF0FBECDBFDF91CF911F91C9
:107100000895CF938091B5038823A1F0C091E90041
:10711000CF709091EC00892F817090FD80E8C82B92
:107120001092E9008091E80083FD0E942137CF7022
:10713000C093E900CF910895DB018F939F930E9444
:107140003739BF91AF91A29F800D911DA39F900DE4
:10715000B29F900D11240895991B79E004C0991FE6
:10716000961708F0961B881F7A95C9F780950895A1
:1071700087FB082E062687FD819567FD61950E9495
:10718000AC380EF4919507FC81950895AA1BBB1BA2
:1071900051E107C0AA1FBB1FA617B70710F0A61B17
:1071A000B70B881F991F5A95A9F780959095BC0138
:1071B000CD01089597FB072E16F4009407D077FDB4
:1071C00009D00E94C63807FC05D03EF49095819501
:1071D0009F4F0895709561957F4F0895A1E21A2EF3
:1071E000AA1BBB1BFD010DC0AA1FBB1FEE1FFF1F6B
:1071F000A217B307E407F50720F0A21BB30BE40BBB
:10720000F50B661F771F881F991F1A9469F7609501
:107210007095809590959B01AC01BD01CF010895BB
:10722000EE0FFF1F0024001C0BBE0790F691E02D0F
:1072300009940E942139332312F48A1B9B0B0C946E
:107240003239A29FB001B39FC001A39F700D811D71
:107250001124911DB29F700D811D1124911D08955F
:107260000E942139B7FF0895821B930B08950E9455
:107270002139A59F900DB49F900DA49F800D911D65
:1072800011240895B7FF0C9437390E943739821BB7
:10729000930B0895FC014150504030F001900616C8
:1072A000D1F73197CF010895882799270895FB01D9
:1072B000DC0104C08D910190801921F441505040AF
:1072C000C8F7881B990B0895F999FECF92BD81BD2F
:1072D000F89A992780B50895A6E1B0E044E050E01F
:1072E0000C949E39A8E1B0E042E050E00C949E3945
:1072F000262FF999FECF92BD81BDF89A019700B46F
:10730000021639F01FBA20BD0FB6F894FA9AF99A0E
:107310000FBE08950396272F0E9479390E9478396D
:10732000252F0E947939242F0C9479390196272F23
:107330000E9479390C947839DC01CB01FC01F99970
:10734000FECF06C0F2BDE1BDF89A319600B40D92B1
:0C73500041505040B8F70895F894FFCF6A
:10735C00C8009802010102001B001B1B01191A1B1B
:10736C001C1D1E1F202122060117311B318F318B52
:10737C003187311A3101F0F1F2F3F4F5F6F700012F
:10738C000203040535343332313690676665E2000A
:10739C00E900EA00B500B600B700CD008301CC00CF
:1073AC008A01920194012102230224022502260261
:1073BC0027022A02B300B4006F007000818283E2BE
:1073CC0000E900EA00B500B600B700CD008301CC9F
:1073DC00008A019201940121022302240225022633
:1073EC000227022A02B300B4006F0070008182836E
:1073FC000001020202020606060909090909090F21
:10740C000F0F0F0F0F15151518191919191919191F
:10741C001919192324406D221312A6118411291154
:04742C0042115B119D
:00000001FF
